:020000041100E9
:10300000002370B5284C0120636101F03DFA402097
:103010000223FE21254A207401F0BCFA002833D196
:103020000223FF21224A207C01F0B4FA00282BD190
:10303000204BA2899A4224D1E3891F4A93420CD1A2
:103040001E4B63611E4B2268002A03D1002B01D066
:1030500023CB23C401F08CFA70BD1A4A934201D0ED
:103060000023F0E7184B194A1B68934205D9C02288
:103070000421207C920001F007FB104B6361144B8C
:10308000E1E700232374EBE7CC223820AC21920146
:10309000207401F0F9FA0028F3D10E4B63610E4B56
:1030A000E3810E4BCFE7C0468463FF1F9063FF1F91
:1030B0009263FF1F5959000083050000E942001187
:1030C00090BA001182150000A863FF1F871300004B
:1030D0009CBA001185430011AAAAFFFF84BA00110F
:1030E000F7B5164B0192C318021D002000938823E8
:1030F0005B05D3181B685C1C1AD09CB2402C18D8F6
:103100008D781E0CAC466746CD782D023D43AE420D
:1031100006D1019800280ED110000C70240A4C70C2
:1031200003249BB20733A343D218009B9A42DED3F9
:10313000FEBD4432F9E71000FAE7C046FC0F00007C
:10314000802213B503000324019189B25201073193
:103150009B18A14304305A1A88235B05C3181B68C7
:10316000591C03D190429241104016BD99B240299A
:1031700007D80B000733A343C0189042ECD30020BC
:10318000F3E74430F9E7134B134A1B68126810B594
:10319000FA24934201D81A00F824104BE4021B6869
:1031A0009A4210D813000E4A12689A420ED3013385
:1031B00007D1F823DB029C4203D10A49054808F0F5
:1031C000BBF8200010BDFC24E402ECE7FE24E4027E
:1031D000F7E7C04600C0071100D0071100E0071153
:1031E00000F00711FFFFFF7FF0B59BB015000490C2
:1031F0000391402A00D9A0E006AB59801A80FFF75E
:10320000C2FF0400042816D9002206A9FFF768FFB0
:10321000052810D906AB1B88AB420CD1002D07D076
:10322000514B2A000499C01808F0CEF9002802D1A9
:1032300001201BB0F0BD06AB1D8020000699FFF7F2
:103240007FFF041E7BD1069B0793FFF79CFF802323
:103250005B01C618802307001B039E4201D3F8269A
:10326000F60288235B05F31801931B68013302D033
:10327000019808F0D9F83D49019808F05DF83B1D28
:103280000293331D05938822029B52059B181B68ED
:1032900008935A1C3CD044219AB20091402A04D889
:1032A0000320D11D814389B2009103991B0C8B42ED
:1032B00024D0402A22D80122300008A9FFF710FFAD
:1032C000021E1BD1380008A9FFF70AFF04000428DA
:1032D00031D9009A059B9B1880225201B218934263
:1032E00040D288235B05C118009A09A808F06CF841
:1032F0001D4B009A09A9F01808F086F8009A029B65
:103300009446634402931A4B029AFB189A42BAD32A
:1033100088235B05FC1821680198013908F00CF836
:10332000200008F081F8039A07AB5A803000079913
:10333000FFF706FF0400002C03D1002079E70428E2
:10334000FBD988235B05E018069907F0F5FF0323F6
:10335000EA1C9A4300D16BE7034B0499E01808F08C
:1033600053F865E70424ECE704000011FFFFFF7F3A
:10337000F80F0000F7B505001400402A21D80027F7
:1033800001AE71803780FFF7FEFE042816D93A009F
:103390003100FFF7A5FE042810D93688BC420BD0B7
:1033A000BD4209D0221CB44200D9321C064B92B255
:1033B000C118280008F008F830B2FEBDC04300B2C2
:1033C000FBE703204042F8E70400001137B5042270
:1033D00004000D0001A81649FFF7CCFF02000428E5
:1033E0000BD1019BA34208D3AB4204D0104901A8E2
:1033F0000195FFF7F9FE01203EBD0E4C2368200029
:10340000019308F011F8019920000139019107F0AA
:1034100093FF80235B01E418074B9C42EED104220A
:10342000034901A80195FFF7DFFE0020E4E7C0464D
:103430005555000000C007110000081130B589B0D3
:1034400008F0CAF910226946254808F0EDF8254B26
:10345000009A9A420ED1019B029A0F2B33D8002179
:1034600001240698013B08D2002900D00292029B59
:10347000013331D10023029325E0551CF2D1020023
:103480002100EFE710341022200004A908F0CCF846
:10349000029B013301D1069B0293882304995B05AB
:1034A000C918059B06981A03120B049105928142D4
:1034B00003D02B4201D107F087FF019B013B019311
:1034C000019B002BDED1029B002B03D004930498B8
:1034D0004168084709B030BDE025014C2D03EFE7F6
:1034E0000000011150485936F7B50F490F4B0A68D3
:1034F00004001A4084235B0013430B60030003277E
:103500001033019300252E00112007F0FDFF084B1A
:103510001B683B40AB4002351E43202DF4D1019B7C
:1035200040C4A342EED1F7BD5CF0004000FEFEFFB8
:1035300064F00040802270B5AD4CAE4BD20000214B
:1035400020001C6008F070F92300AB4A88331A6031
:10355000AA4B1A786E23002A00D01133E3620A23A3
:103560002365A74B1878A74BA0630138E361C3B26A
:10357000032B01D810232362A34B37226361C82396
:10358000DB00A36123008C331A60082336210F3A35
:10359000E518E16323646264E9670439251DE9677E
:1035A00025003B26BC352E602500C0352B6025004C
:1035B000C4352A6025000636CC352E602500083E2D
:1035C000C8352E602500D03529602100D4310B602C
:1035D0002100D8310A6021000225E0310D6025006C
:1035E0004221DC35296025001B3EE4352E60250094
:1035F000E8352B602500EC352A6022000525F432E1
:1036000015602200F03211602200183190321160F2
:1036100022009432136023003C2298331A60AF23B7
:10362000DB002360794B2363032805D808F034F9C5
:10363000330235371523636096232100FA225B009D
:10364000A360E360C8332361714BFC319200A36433
:103650000A6062626F4A704DA2627322E2656D3A3F
:103660006265A2650232E5644A60022161669621C4
:103670008900A166626709210022E166A2676749A5
:10368000674A684E2167E2673560032811D808F061
:1036900003F996089EA61023CDE70E23CBE70C2353
:1036A000C9E720001A259C30056020000735A030AE
:1036B00005602000A83003602300FA20F833800062
:1036C000186023006420A433186023005F38AC33F3
:1036D000186023000338B03318602300C630B433B9
:1036E000186023000020B833186023003825FC330D
:1036F0009D604D4D5A665D644C4D9A64DD61962522
:10370000AD001D624A4D9A675D62F53DFF3D9D62C9
:103710001E25484ADD6618675867D9651966DA6755
:10372000BE23C021444A5B00E250444B4900635031
:1037300004316250C4225200A350FA23E4205B00FB
:103740000432A3500432A3503D493E4A3E4BD1605F
:103750003E49800019503E49E938FF3819503D492B
:10376000043019503C491038D1613C4911633C493F
:1037700051633C4911603C49195019003B48F831EC
:1037800008603B49D16582213A4A89005A501A00A3
:1037900039490832D1671A003849B432116088219A
:1037A000374A89005A501A00364988321160364A21
:1037B000DA6407F001FE012007F016FE70BD20005C
:1037C00014259C30056020000435A03070E72000EF
:1037D00010259C30056020000335A03068E72000EC
:1037E0000E259C30056020000235A03060E7C04601
:1037F0000004FF1F5866FF1F5071FF1F1846FF1F70
:103800004A0AFF1F3A07000080C3C9019A0200005C
:1038100050C300006A180000280A0000204E000073
:1038200088130000F009FF1F00400011681000001D
:10383000C4090000DC05000040420F001027000012
:10384000FD1BFF1FFC00FF1F0000FF1F252FFF1F98
:103850004D32FF1FE530FF1FD91FFF1FF51FFF1F50
:10386000A121FF1F491FFF1FC528FF1F8D2CFF1F10
:10387000D918FF1FD127FF1F3925FF1F4525FF1F1F
:10388000491EFF1F011FFF1FC11DFF1FF7B50B0CB6
:10389000FF270122009300233C001E001D009446D8
:1038A000019089B262469A401000084018413618CB
:1038B000B6B2FF2F02D1012E00D19FB20098024074
:1038C0001A41AD18ADB2FF2C02D1012D00D19CB22E
:1038D0000133102BE6D10320012E07D1012D04D195
:1038E000019B2401E4191C700138FEBD102EFCD18F
:1038F0000238102DF9D00230F7E710B5064C2378C6
:10390000002B07D10548FFF7EFFD0548FFF7ECFD59
:103910000123237010BDC0461866FF1F2C66FF1FD1
:103920001C66FF1FF0B58BB00D000123019010291C
:1039300036D8FFF7E2FF00231A001B48C15C0133B1
:103940005218102BFAD1023B002A29D0174B184CE1
:103950001F68002306A9E25C1600FA5C56405E541C
:103960000133102BF7D102AA07F0AEFF2A0002A9FB
:10397000019807F0B9FD07F0E7FE23681B182360E4
:1039800007F0E2FE63681B18636007F0DDFEA368C2
:103990001B18A36007F0D8FEE3681B18E360002340
:1039A00018000BB0F0BDC0462C66FF1FB844FF1FC7
:1039B0001C66FF1F0223F0B501245F4D5F4E2B7084
:1039C0005F4B91B01C705F4F0393336808207B708E
:1039D00006F06CFA0023984205D07A78552A02D076
:1039E000332A00D09CE03360002006F0DFFC07F0B3
:1039F000C3FCFFF79FFD07F0F7FE1F220124002103
:103A0000514B10AE1A70514B1C70514B1970514BE9
:103A100019689143163A0A431A6060221968914363
:103A2000403A0A431A6007F017FF07F01DFEC12055
:103A3000FF21494B80001A588A431A50C522920030
:103A400098588843BF3901439950985843490840D2
:103A50008021C9010143802099509958C00509026D
:103A6000090A0143995080213D48490107F0B4FDFE
:103A7000032322003B49019400933B4807F054FD87
:103A80002C223A4905A807F09FFC05AC6178207804
:103A9000023406F02BFAA642F8D10121002006F0EC
:103AA00039FB0121092006F035FB314B314A1968F9
:103AB00003201140A022D2020A431A608022196812
:103AC00092040A431A6019682B4A1140802292031B
:103AD0000A431A60294B2A4A934200D8012007F072
:103AE00063FC07F059FE07F0CFFC287807F01CFEB6
:103AF000039B1878C0B207F047FD07F0B5FE2149D7
:103B0000042007F0A9FD06F01DFC00F0AFF800F05E
:103B1000E9FD00F07BFE00F019FA002011B0F0BDC5
:103B200000932100174A042007F08EFC8023DB0558
:103B30009C62FFF783FC57E74A0AFF1F34F00040FE
:103B40001846FF1FB463FF1F480AFF1F490AFF1FE3
:103B5000680AFF1FBCF0004000E100E0FF00FFFF2B
:103B60001C46FF1FA058FF1F1C56FF1FA8B90011BD
:103B700014F00040FF7FF8FFFFFF9FFF5071FF1F11
:103B80000080FF1F3B00010870B500252849294A25
:103B900029484D6308CA1B051B0DED188242F9D157
:103BA0000022264B8B63264B08211A628022254B6C
:103BB0009205DA67244BDA688A43DA60234A12787E
:103BC000012A03D09A6822490A409A600121EE2412
:103BD0002048E40002686C438A430260DA681120DE
:103BE0008A43DA6007F0E0FC112007F065FC112041
:103BF00007F0A2FE184A200C0400642390420AD861
:103C0000FA220023D200904205D9144B0A21C01891
:103C100007F072FCC3B2124A1372124BD4801B78A5
:103C2000002B04D1104B1021187807F045FE70BD11
:103C3000000005408805054000060540FF01000022
:103C400000F0004004E100E03CF000404A0AFF1FA1
:103C5000FFDFFFFF00380040B70B000030F8FFFF28
:103C60009C63FF1FD865FF1FD463FF1F002210B5A0
:103C70001100112007F030FE10BD0000F8B5002340
:103C800001250826394F3A4C3B62E3681120AB43CB
:103C9000E360E368B343E36007F00EFC112007F034
:103CA00083FC112007F0A8FD40232268290013435C
:103CB000236080236268DB02134380226360A36871
:103CC00007201343A360A3682A4A1340A3608023FC
:103CD000A2689B0113431022A360236C93432364C7
:103CE000236C2B43236480235B003B62226B224BBB
:103CF0001A402263626B1A406263A26B1A40A2638D
:103D0000E26B1340E3631D4AE3681340E36006F08F
:103D1000D3F92900072006F0FDF98021184A112067
:103D2000536C0B43536407F0BFFCFD21154B164A3F
:103D300089005A508023C720626B5B03134363637F
:103D4000E36880003343E360E368104A1D43104B8F
:103D5000E56019581140802212020A431A5080224D
:103D600092051A600B4B5E63F8BDC04600F0004040
:103D70003CF00040FFFFDFFFEFFFEFFFFFFF7FFFA3
:103D8000003800400000FF1F893B0011FF00FFFFCB
:103D900000E100E00000054030B503A804880B20D6
:103DA000002C0ED14968074D087849780902014373
:103DB0000A20A94205D1012120001980024B1B7A5B
:103DC000137030BD192A00009C63FF1FF7B5150062
:103DD00008AA16884A680F4F1478527812022243B4
:103DE0000A24BA4214D10122DBB2019200962A00C1
:103DF00007F0F8F9041E0BD1074B1B68002B07D006
:103E000068782A78000210434242504101309847B6
:103E10002000FEBD022900002063FF1F30B50125F0
:103E200003790400BFB02B4212D00A49408806F043
:103E300045FD28420CD06A46074B69465B8D55808C
:103E40001380064B60881B7A1371002203F016FE64
:103E50003FB030BD1863FF1F6042FF1F9C63FF1F10
:103E600010B50549054806F0DFFC0421044A054861
:103E700006F09CFC10BDC0461863FF1FFFFF00004A
:103E8000D4B900116042FF1F10B5024804F078FC5D
:103E900010BDC0461D3E0011062310B583701033BF
:103EA0000371443B43712A3383714433C37100234C
:103EB0000222012103720E4B027041701C88817234
:103EC0004472197A0273C1729A784273DA788273F3
:103ED0000322C2731A7902745A7942740C228274D2
:103EE0009A79C274DB7903751123C370152010BD54
:103EF0009C63FF1F10B5142007F02EFB124B1422F9
:103F00000021186007F090FC002007F02DFA012036
:103F100007F0AAFA022007F0D7FB032003F0D4FE33
:103F2000042005F0E9FE052003F012F9062003F055
:103F3000DFFD072001F074F9082006F017FC0920C6
:103F400000F056FF10BDC0462463FF1F10B507F0F8
:103F5000EBFC012007F098FB07F06EFA002010BD83
:103F6000094B10B50400984205D0012904D1200066
:103F7000064906F059FC10BD0229FCD1013904F0B4
:103F8000BDFB0028F3D0F6E7FEFF00004A63FF1FE9
:103F900030B5012503790400BFB02B4222D012496D
:103FA000408806F08BFC28421CD06A460F4B104913
:103FB0001B8813800F235380243313716B460A220E
:103FC000581D07F001FA6A4669460A4B1B68D3730D
:103FD0001A0A0A741A0C1B0E4A748B740022608829
:103FE00003F04CFD3FB030BD4A63FF1FFE42FF1F90
:103FF0009C63FF1FC463FF1F70B50D7A100004AAF5
:104000002C00168810221440154220D1002E20D1F9
:104010000A78022A18D14A68517815780E4A09029E
:104020002943914205D00D4A914209D01C800A24AF
:1040300004E014220A491A8007F0C6F9200070BD76
:104040000C2208491A80F7E71C800124F6E70824AF
:10405000F4E70B24F2E7C046F3FF0000F4FF000092
:104060009C44FF1FB4BA001110B50400074908486A
:1040700006F0DAFB074804F0C3FA0020E40704D591
:104080000721054A054806F091FB10BD4A63FF1F52
:10409000FFFF0000613F001118BA0011A442FF1F8A
:1040A00000B50C4BBFB01A780B4901A800F0E0FB3B
:1040B0006B4680B25880002809D06A46074B694693
:1040C0001B881380064B0022188803F0D7FC3FB0F2
:1040D00000BDC0462863FF1F2963FF1FFE42FF1F6C
:1040E000FE43FF1F00B50C4BBFB01A780B4901A867
:1040F00001F00AFC6B4680B25880002809D06A465D
:10410000074B69465B8D1380064B0022188803F02D
:10411000B5FC3FB000BDC0465263FF1F5363FF1F95
:10412000A442FF1FFE43FF1FF7B50E00377A1C00A5
:1041300008AB11003D001A8820231D401F423CD1CE
:104140003378022B3BD173681F785B781B023B43AB
:104150001E4FBB4208D01E4FBB4214D01D4DAB4278
:1041600021D00A252800FEBD002A2AD1142C2AD8E5
:104170002200F06807F028F9174B1C70012CF1D9C8
:10418000FFF7B0FFEEE7002A1BD1202C1BD822003E
:10419000F06807F019F9114B04211C70104B1878C6
:1041A00007F08AFBDEE7E3B20124009201940A00E3
:1041B000310007F017F80500D4E70825D2E70125FC
:1041C000D0E70B25CEE70D25CCE7C046F3FF000076
:1041D000F4FF0000022900005263FF1F2863FF1F45
:1041E000D463FF1F10B5024804F0CAFA10BDC046E0
:1041F000913F001170B5160004AA148805AA15781D
:104200004A685078117800022A4A08438018052825
:104210004BD807F041FB03131E29343F0720042C21
:104220000BD80522121BAA4200D92A0022491A8063
:104230003000091907F0C8F8002070BD0720112CC4
:10424000FBD81222121BAA4200D92A001B491A804D
:10425000EEE707200E2CF0D80F22121BAA4200D93D
:104260002A0017491A80E3E70720032CE5D8042227
:10427000121BAA4200D92A0012491A80D8E7072047
:10428000032CDAD80422121BAA4200D92A000E49B4
:104290001A80CDE70720032CCFD80422121BAA4294
:1042A00000D92A0009491A80C2E700220A201A8090
:1042B000C3E7C046DCD5FFFF63BA00117063FF1F80
:1042C00053BA00114EBA001149BA001144BA001194
:1042D00010B50D21024A034806F068FA10BDC04629
:1042E00038BA00111443FF1F37B5002000F0CCF896
:1042F000204D214BEA89287C9A422AD1042201A927
:1043000000F076F9040000F033F9002C30D16B4650
:1043100099882B68C9BA4B432989184A1B145B1822
:1043200053806B46D9886B6849BA89B24B43698917
:104330001B0C5B181248191C1BB2834200DD011CC8
:104340000B0400D5002113889180013313802000D5
:104350003EBD0223002101AA00F01CF96A460400B8
:1043600002230121287C063200F014F90443CAE735
:104370000124ECE78463FF1F830500009C63FF1F9B
:104380000F27000037B5012000F07EF81F4D0722EF
:104390006946287C00F02CF9041E33D16B461B784B
:1043A0007F2B2FD800F0E4F86B46D878F023020476
:1043B0001B031A406B469B8815495BBA9BB21A4394
:1043C0002B68000953432A891B0C9B184B806B46B2
:1043D0005A789B7812031B011A436B6802435343BC
:1043E0006A891B0C9B180B481A1C1BB2834200DD08
:1043F000021C130400D500220B888A8001330B8035
:1044000020003EBD00F0B4F80124F9E78463FF1FEB
:104410009C63FF1F0F27000010B50F4C237C002B5F
:104420000CD0382B0BD1012000F02EF8CC22AC217F
:10443000207C920100F028F900F09AF810BD074B9B
:10444000E2899A42FAD1012000F01EF80021207C76
:1044500000F0FAF8F0E7C0468463FF1F8305000010
:1044600010B5084B1A7C002A09D05B69002B06D0D6
:104470009847041E01D0FEF7C3FD200010BD0124A3
:10448000F9E7C0468463FF1F70B5002106001620BF
:1044900005F076FE0121152005F072FE07F0ACF85C
:1044A0000400092007F0A8F900222B4B2B4DDA66F7
:1044B00061321A6019685B3A9143002E28D0023AA3
:1044C0000A431A60AC4209D10A22DA6107321A6241
:1044D00000221A639A630132DA6370BD204A944263
:1044E00003D11E22DA610532F1E71E4A944203D15C
:1044F0003022DA610632EAE71B4A944203D14322B2
:10450000DA610832E3E7194A9442E1D16922F7E718
:1045100002220A431A604622AC4203D0104A944257
:1045200004D194225A6106329A61D1E70D4A94422D
:1045300001D1E622F6E70C4A944204D13422FF323C
:104540005A610D32F0E7094A9442C1D1E622520085
:104550005A610A32E8E7C046005000400024F400E7
:104560000048E801006CDC020090D00300D8B805D8
:1045700010B50024064B0920DC6606F09DFF2100E3
:10458000162005F099FD2100152005F095FD10BDC0
:1045900000500040F8B51C000023134D0F00EB66DF
:1045A0006860160007F018F901238022EB662300EB
:1045B0002F615200013B08D206F0A6FE08200B4AEC
:1045C0001168002C03D12000F8BD2A61F2E72B6F9F
:1045D000034203D02B69013C3370013613685B1A28
:1045E000032BEED90124EEE7005000406008FF1FC6
:1045F000002370B5124D1400EB6668600E0007F0E2
:10460000EBF801238022EB6623005200013B08D225
:1046100006F07AFE08200B4A1168002C03D1200016
:1046200070BD2A61F2E72B6F034203D02B69013C76
:104630003370013613685B1A032BEED90124EEE7C1
:10464000005000406008FF1F002370B50C4C0D00A7
:10465000E366606007F0C0F80123E366256106F0B9
:1046600053FE8020074A80001168636B034205D126
:1046700013685B1A032BF8D9012070BD0020FCE7FA
:10468000005000406008FF1F002370B5134C0E005F
:10469000E3666060150007F09FF80123E36626617A
:1046A0000F33626B1A42FCD02B0A23611023626B1A
:1046B0001A42FCD0EDB2256106F026FE8020084AA1
:1046C00080001168636B034205D113685B1A032BEA
:1046D000F8D9012070BD0020FCE7C0460050004022
:1046E0006008FF1F10B5084CE368002B08D1074B8A
:1046F0001B685B045B0C0A336360054B1B6823601B
:1047000006F00AFFA06010BDC463FF1FC8F00040A0
:10471000CCF0004010B507F05FF80F4B996A9A6A29
:104720008A42FBD10D4C6268A0688A18121A531E87
:10473000884200D31300A1602168DA0B52185B0491
:1047400007495B0C636022600B60064B1A6006F041
:10475000DBFD206810BDC04600F00040C463FF1FB1
:10476000C8F00040CCF0004070B51F4C23793F2BBF
:1047700001D93F2323711D4B22791A701878C0B2DA
:1047800006F07AFF18231A491A4A0B801A49138037
:104790000B805380A379194980200B800C219380D2
:1047A00001334B430001191C834200D9011C144BF7
:1047B000D18019806379002B11D101336371237A81
:1047C000012B01D8022323726279237A0D485343C7
:1047D0000A21584306F090FE0B4D286070BDA02BB7
:1047E000EDD9A023EAE7C046B863FF1F480AFF1FC0
:1047F000FC43FF1FC445FF1FFA43FF1FA465FF1FB3
:10480000F843FF1F71020000A863FF1FF8B51221D3
:104810000020FEF7DBFD114C011E114D09D10C22C9
:10482000104BC1CBC1C4280006F0FEFFFFF79CFF70
:10483000F8BD0C2220000C49FEF79CFD0C2802D08C
:10484000084B43CB43C40C2228000849FEF792FDD5
:104850000C28EBD00C220021E5E7C046B863FF1F0F
:104860008463FF1FA8BA0011FC0C0000F50C0000C7
:10487000F0B5002604000D0085B0B24262D04B1C9A
:10488000087801934B7889782F7909021943EB78DE
:104890003F061B040B431F430397207066702528B7
:1048A00000D172E012D810280AD806F0F5FF45E6CC
:1048B0002B2B2B86948D2B2B2B2B2B2B2B2BC600B2
:1048C000232800D1A8E0FF23637093E0562856D038
:1048D0000FD8332800D198E0552836D02628F2D1B9
:1048E000934D13223100280006F09EFFFEF788FB4F
:1048F0005AE0722800D17FE0DC2800D1DCE071288A
:1049000000D16FE0DB2800D0F1E0042ADBD91026CB
:10491000052A05D0561F32003800691D06F054FDE7
:1049200005222900200006F04FFD32003900601DED
:1049300006F04AFD053605E00C2220007D4906F010
:1049400043FD0C26300005B0F0BD013A7A4D0C2A2B
:1049500013D8002A0AD02800019906F035FDFFF788
:1049600003FF0C2228007549FEF73EFC0C222900AB
:10497000601C06F029FD0D26E4E70C22EBE76E4DE6
:104980006F4B2A0043CB43C2E9E7013A684D0C2A3A
:1049900011D8002A08D00199280006F015FD0C2234
:1049A00028006849FEF720FC13222900601C06F04D
:1049B0000BFD1426C6E70C22EDE705226249601CB8
:1049C00006F002FD0626BDE712226049601C06F0D3
:1049D000FBFC1326B6E708225D49601C06F0F4FCD8
:1049E0000926AFE76978F72900D96CE7594B188891
:1049F00001F0E6FB0226A5E7574B012A03D06A78AF
:104A00001A706270F6E71B785EE70A225349601C51
:104A100006F0DAFC0B2695E7042A04D9504D2F60E6
:104A200006F07AFDA860FFF775FE0422039003A943
:104A3000601C06F0C9FC052684E74A4D062A15D9F4
:104A400006222800019906F0BFFD00280ED006229C
:104A50000199280006F0B8FC062243492800FEF719
:104A6000C3FB01233C4A11780B4313700622290033
:104A7000601C06F0A9FC072664E7931E3B4F1A2B27
:104A800004D86B78002B09D100F026F9384B390097
:104A90001E78601C721E06F097FC53E7551E2A0014
:104AA0000199380006F090FC3249AAB23800FEF7AE
:104AB0009BFB00F047F9E9E7022A00D803E76B788F
:104AC000BFB26370AB78A370032A05D0033A3900F4
:104AD00092B2E81CFEF788FB10223900E01CFEF7BA
:104AE00049FCC61C002800DB2CE7607082E7DA284E
:104AF00000D0E8E6042A00D8E5E6082A15D9AB7903
:104B00006A791B021343EA7912041A432B7A1B06B3
:104B100013433B603B68052229002000039306F005
:104B200053FC0422601D03A958E7FE236370F1E7DC
:104B30008463FF1FB4BA0011B863FF1FFC0C0000B0
:104B4000A8BA0011F50C00009063FF1F7063FF1FEF
:104B50003845FF1FFE43FF1FB463FF1F9C63FF1F09
:104B6000C463FF1F6509FF1FADAC0000B765FF1FE1
:104B7000B565FF1FAEDE000070470000020010B5F3
:104B8000094B0A32094C92B2DA815A829881188212
:104B9000207802F07BF90422054B012120781A705D
:104BA00006F08AFE10BDC046C244FF1F0266FF1F0A
:104BB0000166FF1F013870B5042809D806F06CFEA5
:104BC0000309210812001D4B0221187806F074FE1B
:104BD00070BD1A4B0821187806F09EFB0022184B76
:104BE0001A72F5E70024164B144D082128781A682C
:104BF000DC721C8106F000FC2100287806F07CFDA8
:104C0000E6E70E4B0821187806F086FB0D48FFF703
:104C100043F90D4B0D4A9B7993800D4A1380002276
:104C2000074BDA720132FF321A810A4B1B78002BD4
:104C3000CED0094A136006F0FFFCC9E7D463FF1F1A
:104C4000A863FF1F0744FF1FB863FF1FC445FF1F72
:104C5000A465FF1FB463FF1F34F0004010B50029A6
:104C600005D1082803D10131013005F053FA10BDF8
:104C700010B501290FD108280DD10021013005F010
:104C800049FA054B1B78002B05D02622034B04481C
:104C90005A72FFF773FF10BDD865FF1FA863FF1F8F
:104CA000C40900000300F0B50A4D8E18B14202D1CC
:104CB00052008018F0BD0C782F6824093C5D0F2746
:104CC0001C700C7801313C402F683C5D5C700233F5
:104CD000ECE7C046F443FF1F0E22114B10B51A70CB
:104CE0000D23104C10492370093A043B0F486370A0
:104CF00006F06AFB2D2301220D490E48E371FFF7F0
:104D0000D1FF01220C49FFF7CDFF01220B49FFF72C
:104D1000C9FF00220A491000FEF766FA10BDC0461E
:104D2000D465FF1FB565FF1F63BA0011B765FF1F8C
:104D30006709FF1FBD65FF1F6609FF1F6509FF1F8C
:104D4000AEDE000070B5124C132220001149FEF7B0
:104D500011FB114D002817DDAB78002B14D0431C3C
:104D60002B7009236B700023001903702878290029
:104D70000130C0B206F050FC297822000139C9B2D6
:104D8000002005F031FC70BDFFF7A6FFEEE7C0463E
:104D9000B765FF1FAEDE0000B565FF1F10B5114BF4
:104DA0001A781870002A0ED000280BD10E4B1A78F2
:104DB000062A07D85423D340DB0703D50B4B1878BA
:104DC00002F064F810BD0028FCD0074B1B78012BC3
:104DD00002D0033B022BF5D8044B0121187806F0D2
:104DE0006BFDEFE7D865FF1F0166FF1F0266FF1F1F
:104DF00070B5504E504A51493070082005F080FA85
:104E00000121092005F086F9092005F067FA012142
:104E1000002005F07FF9002005F060FAFEF7F0F8B9
:104E200006F0BAFB032246494648FFF73BFF2D2414
:104E3000030004221C7044490130FFF733FF302384
:104E40000470424D424C437083702E3B062220007A
:104E50004049EB87FEF78EFA062813D0200006F0B3
:104E60004BFD022809D00321200006F0CDFB8D2345
:104E7000E3706E3B237119336371062220003549BC
:104E8000FEF7B2F9344B1B68FC335C64FFF75AFF42
:104E90000020FFF783FF314C314A0121314B12785A
:104EA000207801F0B5FF304A304B1278002120788D
:104EB00001F0AEFF01222E4B1A702E4B5B78552B62
:104EC00031D12D4B3B325A722C4B2D4AAB81EA81AA
:104ED0002B826A822021307806F0E6FC01204042D5
:104EE00005F0CEFB0120404205F06AFCFFF7F0F927
:104EF000FEF7B6FF00F0A0FC01204042FFF7B4F837
:104F0000012006F001FCF72001F03EF90121307884
:104F100006F0D2FC307802F015F91A4806F05CFA77
:104F2000FEF7ACFE70BD6422174B5B7953431A0049
:104F30000A32CBE7D463FF1F5D4C0011714C0011A6
:104F40003845FF1F7063FF1F9063FF1FC244FF1FA0
:104F50006509FF1FADAC00005866FF1F0266FF1F0A
:104F60002644FF1F0744FF1FD465FF1FB565FF1FC1
:104F7000A665FF1FB463FF1FA863FF1FC4090000DD
:104F8000CE090000D663FF1FB863FF1FF8B50A0003
:104F900020230D001A40194251D0544B1B78002B8E
:104FA0003CD0FFF7B7FB524B524C534E99686268A6
:104FB000737A8A1ADB039A4202D36160FEF75EFEBF
:104FC000327A217A531EDBB299422AD1FFF724FAB2
:104FD000637A002B1FD0013BDBB26372002B1AD126
:104FE000464B5B78552B01D106F026FBE37A002B6C
:104FF0000CD00023424A434FE37213883800013338
:105000001380FEF749FF390006F04EFA64237079E9
:105010005843FFF7B3FD237A013323722020684001
:10502000F8BD9142D4D300232372FFF719FA354F0C
:105030003800FEF731FF390006F036FAC8E70BB248
:10504000002B0ADA304B187806F07EFC002801D0DD
:1050500006F082FB80200002E1E70224214206D014
:10506000244B01201A72FFF799FE2000D7E70B07A7
:105070001BD5FFF74FFB1E4B1E491F4C98684A6813
:10508000637A821ADB039A4202D34860FEF7F6FD88
:10509000FFF7E6F9FFF7C0F900F0E8FB2368DB074C
:1050A00001D5FFF79FF80820B9E710240E0026402D
:1050B000214206D00D4B1B78002BD6D1FEF7E4FE23
:1050C000D3E70124214209D0104800F06DF806F022
:1050D000B3FB3100092005F01DF8C6E704240800E1
:1050E000204021429CD0FEF7DBFFBEE7D865FF1FC2
:1050F000C463FF1FA863FF1FB863FF1FB463FF1FD4
:105100009C63FF1F0744FF1FD463FF1FEC43FF1F77
:10511000F0B51B4B1B4F1B883A8804001A4E1B4DE1
:1051200085B09A420DD832889A420AD3184B1A8811
:105130002B889A4205D1174A174B12881B889A422E
:105140001BD0052001F076F83B8802AA1380338833
:10515000019053802B88114D93800F4B02A91B881F
:10516000D3800F4B2A78188802F092FD0D4B08214E
:105170002878019A1C7006F007FC05B0F0BDC04607
:10518000A265FF1FFC43FF1FFA43FF1FA465FF1F1B
:10519000A065FF1F9E65FF1FF843FF1F0266FF1FEC
:1051A000FE43FF1F9C65FF1F13B50C4B1C78002CA2
:1051B00011D1002801D00A4B18600A4A0A4B117815
:1051C0000A4A10780A4A01920A4A0092002205F01F
:1051D00003F9200016BD1124FBE7C0460166FF1F3E
:1051E0009865FF1F0066FF1FF065FF1F0266FF1F27
:1051F000DC65FF1FE065FF1F10B5064B12201B7812
:10520000052B06D1044B13221988044B187801F0A2
:10521000EDF910BD0166FF1FFE43FF1F0266FF1F71
:1052200010B500240122114B52421870104B1C7013
:10523000104B1A8001F086FF04220F4B21001A70D8
:105240000E480C3206F028F9102221000C4806F016
:1052500023F907220B4B1C600B4B1C700B4B1C7073
:105260000B4B1A700B4B1C7010BDC0460266FF1F23
:105270000166FF1FFE43FF1F0066FF1FF065FF1F53
:10528000E065FF1FDC65FF1FB465FF1FB365FF1FEF
:105290000044FF1FB265FF1FF8B5174C06002578C4
:1052A00006A814240078052D23D1B41F134FA5B2EE
:1052B0001824BD421DD88D1FADB2BD4219D8FA25A4
:1052C0006D00AA4215D21D000D4F0A3DADB2BD4280
:1052D0000FD80C4C26800C4C21800C4900240A80ED
:1052E0000B4A1380FFF714FF0A4B0421187806F0CD
:1052F00013F82000F8BDC0460166FF1F790C0000BE
:10530000750C0000FC43FF1FFA43FF1FA465FF1F3D
:10531000F843FF1F0266FF1FF0B50BB20D0089B006
:10532000002B00DB70E1A44E307806F00DFB041E6C
:1053300050D00378A22B00D122E1D02B1AD0912B90
:1053400045D143780E2B42D19C4B82889A423ED164
:105350009B4A83681278052A39D1032018567F2882
:1053600035D0984B1B68002B31D05B68002B2ED0BA
:1053700098472CE08078072829D806F08DFA042871
:10538000183F3F74A8D86378002B0CD101218C4BB7
:1053900019708D4B1A78002A5BD08C4B307801F055
:1053A00037FD002855D00722854B1A7051E06178EF
:1053B0000029F8D1E378002B11D0854A854B12786B
:1053C000307801F025FD60706378002BEBD1200070
:1053D00006F0C2F980200002684009B0F0BD784BA9
:1053E0001B78022BF3D00121307806F075F80028E5
:1053F000EAD10121307806F05FFAE5E76378002B07
:10540000D1D16F4F032807D13B78052B02D101334F
:105410003B701EE00223FBE76F4B1A886F4B029331
:10542000002A0BD01B78002B03D00121307806F026
:10543000ABFA3B78062B04D1013BE9E7029B1A70DB
:10544000F7E7042B41D10121029B3078197006F057
:1054500033FA5C4B1B68002BB9D01B68002BB6D00D
:10546000574A107884E76378554F002B27D10622DE
:10547000211D5B4805F0A8FF62895A4B5A491A80E2
:10548000A2895A4B1A80E3890B800521397058494B
:105490000A80584A1380228A574B1A80574B1B7830
:1054A000012B09D11F2000F0C5FEFA2292004243D1
:1054B0000421307806F068FA0022484B75E7312B5A
:1054C00000D070E70022454B1A700323A0E70622A4
:1054D0000021434805F0E0FF0023454A04211380E2
:1054E000444A30781380444A138005F015FF0821A0
:1054F000307805F011FFA379083B5A425341304AF6
:1055000003331370304B1B78002B06D0334B3078AD
:105510001A78002A06D001F0B9FC0122314B524220
:105520001A8096E70121197006F0C6F9F5E70821FF
:10553000307805F0F1FE6378002B00D047E72C4B64
:105540002D4F0293E388029A04211380294B30786F
:1055500003932389039A138063893B8005F0BCFF82
:10556000002800D033E7264B1B68002B00D12EE724
:10557000039902983A88098800881B68984726E7AB
:105580004379132B00D022E70389012B0AD11D4B4D
:105590001B78022B06D10821307805F0BDFEFFF7FD
:1055A0002BFE14E7052000F045FE082102003078AC
:1055B00006F0EAF90BE7C0460266FF1F051400007B
:1055C0000166FF1F9865FF1F2644FF1F0744FF1F4A
:1055D000D465FF1FB565FF1FD665FF1FD865FF1F88
:1055E000A765FF1FFE43FF1FAE65FF1FB065FF1FCE
:1055F000A265FF1FA065FF1F9E65FF1FA665FF1F19
:105600009465FF1F9C65FF1F8020C001014200D0F0
:10561000E2E6CB0731D5324B1B78002B1DD0314E43
:1056200005AC3378052B1AD1023B23702E4B210099
:105630001B7823722D4B1B7863722D4B187801F069
:105640008BFB002809D007202A4B30701B68002BE9
:1056500003D01B68002B00D098470120BCE60E2029
:10566000254B06221B7825492370254B1B78637038
:1056700002ABC01805F0A8FED8E7022308001840C6
:10568000194209D0174B1B78052B03D11D4B1888E5
:1056900006F02AF802209FE60424214203D0FFF7F7
:1056A00037FD200098E6082308001840194200D171
:1056B00093E6154B1C78012C03D0022C0DD008204A
:1056C0008AE6124B124A134913481B88128809882C
:1056D00000880094FFF7E0FDF1E7FFF78DFDEEE7AE
:1056E000D865FF1F0166FF1F0044FF1FB265FF1F43
:1056F0000266FF1F9865FF1FB465FF1F0144FF1F6F
:10570000B365FF1FFE43FF1F9C65FF1FF843FF1F8C
:10571000A465FF1FFA43FF1FFC43FF1F10B502A83B
:1057200004880B20002C10D14968087849780902B8
:1057300001430C48814209D1022119800A4B598842
:105740001170DB7800205BB2537010BD074C0A204B
:10575000A142FAD102211980034B998811705B791B
:10576000F0E7C0466E2A00009C63FF1F6F2A00000E
:10577000F7B5150008AA16884A680F4F14785278B2
:10578000120222430A24BA4214D10122DBB201924E
:1057900000962A0005F026FD041E0BD1074B1B685E
:1057A000002B07D068782A7800021043424250410B
:1057B000013098472000FEBD022900001466FF1F3B
:1057C00030B5012503790400BFB02B4227D015491D
:1057D000408805F073F828420DD06A46124B69469E
:1057E0005B8D138002235380104B5B88938060880D
:1057F000002202F043F90E49608805F05FF8C00707
:105800000DD56A460B4B69461B88138002235380D3
:10581000064B9B8893806088002202F02FF93FB0EE
:1058200030BDC0460C66FF1F2844FF1F9C63FF1F4E
:105830000466FF1F8244FF1F10B5074C0749200074
:1058400004F0F2FF2000064904F0EEFF0721054AAC
:10585000054804F0ABFF10BDFFFF00000C66FF1F02
:105860000466FF1F34BB00112844FF1F10B5024817
:1058700002F086FF10BDC046C15700110200F0B50E
:1058800001270A480A4E51188B1A002B00DCF0BD84
:10589000082415784308684038404000805B013C8C
:1058A00058406D08002CF5D10132EDE7FFFF0000F4
:1058B0004EBB0011F0B500250F269D4200DBF0BD68
:1058C0004C5D070944403440A400A058013578409D
:1058D000F3E70000F0B589B06A460D000B000F2712
:1058E000110010351C780133260024093E40167043
:1058F00054700232AB42F5D12023024AFFF7DAFF9F
:1059000009B0F0BD54BB0011F0B54E780B7889B0EA
:1059100036020C00170001901E43012A61D9954BF5
:105920009E4200D877E001339E421CD1062A17D14F
:10593000CA788B7812021A430B791B0413434A79F5
:1059400012061A438C4B5A6100221A705A808B4AF5
:105950005A608B4A9A608B4ADA60002009B0F0BD29
:1059600088225205EEE7884B9E423CD182498B78D3
:10597000002B00D0F6E00C2A31D10F22A3789343FC
:10598000E278120213432279120413436279120659
:1059900013434B60E279A07912020243207A00049B
:1059A0001043627A12060243CA60E27AA07A1202B7
:1059B000024376484A81834208D804236E49142260
:1059C00001980B7005F000FD1420C7E71201D218F2
:1059D00089235B059A42F0D801238B70BDE7022A28
:1059E000FAD00523EAE76A4A01239642E6D1FFF797
:1059F00003FC052F0CD9E378A2781B02134322790C
:105A000012041A4363791B061343624A039313601B
:105A100005F012FEA1E7584D2B78002B9DD1AB78F5
:105A2000002B00D1A0E02B8901339BB20093B3423D
:105A300000D091E0132AD4D9CF7C8B7C3F02122175
:105A400020001F43FFF71AFF874200D08EE0002E90
:105A50003DD1E378A2781B0213432279E96812044E
:105A60001A4363791B06134303930A228B4212D114
:105A7000FF23A370E370237163716B89002B09D13D
:105A8000E37B227C1B0212041343A27B13431B09FA
:105A900001336B8100226B89002B8ED0002A67D1E5
:105AA000686837013818000B6B690003039098424F
:105AB00005D9686105F0B8FCEB780133EB706868D4
:105AC0001022A11C381805F09FFC2E8145E76F8934
:105AD000009A7B1E9BB293423AD1E278A3781202DD
:105AE0001A43237905A81B04134362796C681206D4
:105AF0001A43EB6800920392211D0C22049305F0D7
:105B000063FC0120260004A940421036FFF7E2FEA4
:105B1000013F012F17D1009A0B232861824200D048
:105B20004CE704221C49200005F06EFC042203A966
:105B3000686805F001FDE968039AFF23914200D1EE
:105B40003CE7F73B3AE73100FFF7C4FE1036DFE7EA
:105B50000923B742A4D831E7009BB34200D9FCE641
:105B600007232BE7022329E7032327E7062325E75B
:105B70000A2323E7FFFE00009C44FF1F00000111E1
:105B8000FFFF00005048593601FF0000FFFF0011E1
:105B900002FF000034F00040A844FF1F10B5034C82
:105BA0000B000122210000F06BFA10BD5D5D0011B9
:105BB0000B8870B506000D000224162B11D92B009E
:105BC0000322094900F05CFA041E0AD1074B2A8817
:105BD0001B88191C934200D9111C300089B200F0B7
:105BE000EFFA200070BDC046895D00117266FF1F8C
:105BF00010B54A780400013A0B000220012A07D8A8
:105C00000A78002A04D005222000024900F038FA60
:105C100010BDC046B75D00110A7810B50B00040036
:105C20000220002A04D007222000024900F028FAAE
:105C300010BDC046635E00110A7810B50B00040069
:105C40000220002A04D009222000024900F018FA9C
:105C500010BDC046C95E001110B5034C0B000B22ED
:105C6000210000F00DFA10BDF95E001110B5034CD3
:105C70000B000D22210000F003FA10BD6B5F001134
:105C800010B5034C0B000F22210000F0F9F910BDF4
:105C9000C55F00110A7810B50B0004000220002A2D
:105CA00004D011222000024900F0EAF910BDC046DC
:105CB000D55F0011002310B51322190000F0E0F9A0
:105CC00010BD000010B5034C0B001722210000F09E
:105CD000D7F910BD27600011002310B51922190053
:105CE00000F0CEF910BD000010B5034C0B001B22D4
:105CF000210000F0C5F910BD61600011F7B584897D
:105D00000D0006000121002C22D000238268D3560A
:105D10001778002B1EDA0C2C1AD90C3CA4B21319DC
:105D200040880093230002F086FE431E9841013014
:105D30007B06DB0F6B703F23013C1F40A4B2287031
:105D4000AF70AC80002C07D0B3680133AB6000218A
:105D50000800FEBD0020EBE7AC60F8E70B780370AD
:105D60004B8843704B881B0A83700B79C3700420E7
:105D700070470420022B06D10020537811781B02B3
:105D8000009A0B43138070470B8803700B881B0A23
:105D90004370022070470420009983420AD153784F
:105DA00010781B0203430B80D37890781B020343C7
:105DB00000204B807047F8B50D004B78012400217E
:105DC000461C03702B788B4201D82000F8BD6B78FD
:105DD000B01C4F1C012B10D1890069184B8802227E
:105DE00033704B88B9001B0A7370691805F07CFB8F
:105DF00004360434A4B2F9B2E4E7122359436B1811
:105E00005A88043132705B8810221B0A737069183B
:105E100005F06AFB12361234ECE770B5049D1400ED
:105E20001E00052B01D8042070BD637812781B0278
:105E300013432B80E378A2781B02134302226B806A
:105E40002A71211D681D063E05F04EFBB2B22A8163
:105E5000F02AE8D82800A11D0A3005F045FB0020F3
:105E6000E2E7002310B50A789A4201D8900010BDED
:105E70009A008A185488013304705488DBB2240ACB
:105E80004470948884709288120AC2700430EAE7E1
:105E900010B51100029C062B04D004201022142BF4
:105EA00001D010BD022222714B7808781B020343F7
:105EB0002380CB7888781B02034363800431601D04
:105EC00005F012FB0020ECE710B50C788B7804315C
:105ED0005C43E4B203702200013005F005FB601C56
:105EE00010BD0420022B06D10020537811781B022C
:105EF000009A0B431380704710B50C000A880231DA
:105F000005F0F2FA208810BD70B504000D00049869
:105F10001100012B01D8042070BD167852781202AE
:105F2000324302800200F83255701470E825002CCC
:105F300000D10C35023B9AB24280AA42EBD8023122
:105F4000043005F0D1FA0020E6E7042000998342EE
:105F50000AD1537810781B0203430B80D3789078D2
:105F60001B02034300204B80704710B50C000A88C9
:105F7000023105F0B9FA208810BD000070B501218A
:105F80001E000420049C0E400B4218D1CB40DDB211
:105F90008D4214D90A49DBB2098899420FD32300F4
:105FA000F6331D703300580011184978165C090249
:105FB000314301332152D9B28D42F4D8002070BD53
:105FC000BC44FF1F10B50C000A88023105F08CFAA2
:105FD000208810BD10B50C788B7804315C43E4B296
:105FE00003702200013005F07FFA601C10BD10B56F
:105FF00011000298032B01D8042010BD14785278A8
:10600000043B120222430280CA788C781202224397
:1060100042809AB28280F22AEED80431063005F02E
:1060200063FA0020E9E710B50C000B8803700B88B9
:106030001B0A43704B8883704B881B0AC3708A8885
:106040000430063105F050FAA088043080B210BD4B
:106050000420012B03D100201378009A137070479D
:1060600010B50C000B8803700B881B0A43704A881C
:106070000230043105F038FA6088023080B210BD79
:10608000F0B589B003931E4B029242000700D05A2C
:10609000019102F020F81325061E2DD0029B012449
:1060A0000370019B002B04D0001903999847001935
:1060B00084B26B461B7A5BB2002B0FDA10213800DA
:1060C00002F01CFB1925002813D130003219E1B26F
:1060D00002F066FC051E0CD10C34A4B2042304AA01
:1060E000380005A993800696948101F0AFFD051E46
:1060F00002D0300005F048F9280009B0F0BDC046D4
:106100007066FF1F70B505000C0000280CD0002041
:10611000814209D010222000044905F0E5F9012050
:106120002B7823736B78637370BDC04694BB0011EA
:10613000F0B506000D0017001C0085B002291BD029
:106140000020102907D1022B07D0102B03D115E016
:106150000020102C08D005B0F0BD69463800FFF7CC
:10616000D1FF2A0069460BE069463000FFF7CAFFFD
:1061700022006946380004E0022BE9D12A003900E8
:10618000300005F0E1F9E6E7031CF72800D9F72312
:10619000032008499AB2013A0B80D31703400649FD
:1061A0009B189B100B80D30F04499B185B100B802E
:1061B0007047C046C044FF1FBE44FF1FBC44FF1FC2
:1061C000034B1B888B4202D3024B4000C1527047E5
:1061D000C044FF1F7066FF1F014B4000185A7047F4
:1061E0007066FF1F1722014B1A8070477066FF1FF1
:1061F00070B505000E2005F02FF9041E13D0D02332
:10620000037000230622837007494570033005F0B0
:106210006BF9064B2100DA8A62811B7E2373044BE3
:10622000187805F0C9F970BD8C66FF1F7C66FF1FEA
:106230001045FF1F262803D8024B4000C05A704764
:106240000148FCE7C244FF1FFFFF000070B50600D5
:106250000C00094D1C220021280005F01DF9074BF8
:106260001E70074B1C7005F06FF80123002801D049
:10627000002312202B7070BD7C66FF1F1045FF1F8E
:106280009D66FF1F70B505000D4C0800E260A1601F
:1062900010220021656005F0FFF9012803D11021CB
:1062A000A06802F058FD10220021280005F0F4F942
:1062B000012803D11021606802F04DFD70BDC04679
:1062C0007C66FF1F70B5041E05D1002903D006228D
:1062D0000D4805F009F90D4B1D78012D11D1002C49
:1062E00005D102221A7005F097FA280070BD00222D
:1062F0001A70074B1B78FF2BF7D02000FFF778FFB1
:10630000F3E70025F1E7C0468C66FF1F7C66FF1FA0
:106310001045FF1F030010B5002801D1002010BD5B
:1063200000780B4A002803D15988D1821B79137653
:106330001378022BF2D10023984200D1033313705B
:10634000044B1B78FF2B01D0FFF752FF0120E6E73B
:106350007C66FF1F1045FF1F002911D000280CD0BC
:106360004B79012803D140225242134303E03F22DC
:106370001340032802D001204B7170474022F4E7FC
:106380000800FAE770B5094D0100287800280BD005
:10639000074C0622200005F0A7F821002878FFF717
:1063A000DBFF200005F068FA70BDC0469C66FF1F49
:1063B0007666FF1F00290AD0012808D13F224B79B9
:1063C0009343C02B03D0403B5A425341981C704723
:1063D00070B5174D06002B78FF2B15D00A2005F05D
:1063E0003BF8041E10D0D0230370C83B8370114BC0
:1063F00011491B784670C3700622043005F074F80A
:106400002100287805F0D8F80C4B1B78012B0DD112
:106410000B4B1B68002B03D09B68002B00D09847C8
:10642000084B04211878084A04F0E6FF70BDC04606
:106430001045FF1F9C66FF1F7666FF1F9866FF1FB3
:10644000C466FF1FC866FF1F60EA0000014B986822
:106450007047C0467C66FF1F014BDB6818687047B9
:106460007C66FF1F074B10B5DA68136801331360B1
:10647000054B1878FF2803D08021C90105F01CFACC
:1064800010BDC0467C66FF1F1045FF1FF7B50E000C
:1064900002F0C8F8051E1CD00E4B06621F78002FB4
:1064A00000D10778AB791020019304F0D5FF041ECA
:1064B0000FD0D0230380C73B8370019BE91DC370BD
:1064C0000622043005F010F821003800E66005F0DF
:1064D00073F8F7BD0E45FF1F014B18787047C04693
:1064E0009C66FF1F054B002805D1054B1A78054B0C
:1064F000002A00D1014B18007047C0468C66FF1F70
:106500009C66FF1F7666FF1F014B58687047C046A8
:106510007C66FF1F024B1868431E9841C0B270474B
:10652000A066FF1F421E03000120152A03D9FF3B6E
:106530005A425341D8B27047F0B51C0000230E00F8
:1065400085B0039002920B70029A934201D300200F
:1065500019E0E55C5A1CD2B2002DF8D0029851190E
:106560008142F4DC0233DFB2A35C18000193FFF731
:10657000D9FF002807D0013D019A0399EBB233708F
:106580008A4202D1E01905B0F0BDDB19DBB2DBE7CE
:1065900010B50C0002F09EF803001220002B03D06F
:1065A0002100588805F0C8F810BD000070B50E4DE8
:1065B00084006359002B15D0186A002801D005F01B
:1065C00003F92B59586A002801D005F0FDF82B5922
:1065D000986A002801D005F0F7F8285905F0F4F87A
:1065E00000232B5170BDC046AC66FF1F1C4B70B51D
:1065F00004000E00150099420AD11A4B1B68002BAB
:1066000001D1122070BD1B68002BFAD09847F9E722
:10661000154B994215D1134B1B68002B0AD01B68F0
:10662000002B07D09847002804D1104B1C70104B4A
:106630001D70E7E729002000FFF7AAFF0028E1D13D
:10664000F3E7080001F0EEFF0028DAD0037803201A
:10665000A342D7D12900300005F06EF8D2E7C0463A
:10666000FEFF0000A866FF1FFFFF0000A566FF1FDA
:10667000A466FF1FF7B50400808801F0D3FF002552
:10668000A84203D00578A08802F008F81C4E3378A1
:10669000002B1FD0AB421DD11A4B28001978FFF7F1
:1066A00077FF002818D000233370A3790820A7783B
:1066B000A688019304F0D0FE011E0DD0D0230370F4
:1066C000CA3B8370019B477086808371280004F069
:1066D00073FF01E0002DE8D1A0880B4B8200D35856
:1066E000002B01D0FFF762FF1721A088FFF768FD9C
:1066F000A08801F027FDA08801F0FEFDF7BDC0468F
:10670000A566FF1FA466FF1FAC66FF1FF0B587B02C
:106710001D000CAB1B88070001930DAB1B881420D8
:1067200002930EAB1B88160003930FAB1B880091DE
:10673000049310AB1B88059304F08EFE041E1AD040
:10674000D0230370CB3B47708370C67006222900AC
:106750000430002D11D004F0C7FE019B210063819D
:10676000029B0098A381039BE381049B2382059BEA
:10677000A37404F021FF07B0F0BD04F08DFEECE738
:10678000F7B5009308AB1B8807000C200D0016001E
:10679000019304F061FE041E13D0280001F042FFB3
:1067A00000280FD00078D0232370C93BA370009B32
:1067B00021002381019B6770A580E680638104F03E
:1067C000FBFEF7BD014B1878EDE7C0461045FF1FF3
:1067D00013B5040064890389C2888188C078009455
:1067E000FFF7CEFF13BD000010B5044C2068002851
:1067F00003D004F0E9FF0023236010BDB066FF1F43
:10680000A122F0B5818892004A43384B384F1B686B
:1068100004009B189D2292009B18827989B01A600F
:106820003B68002B5FD01D78324B1B68002B04D0D7
:106830005B68002B01D00020984726000836310005
:10684000E079FFF7B7FD237DE0710200E078049363
:10685000638A29000393238A0293E3890193A3881F
:1068600000933300FFF752FFE378002B0BD1E2894E
:10687000A379A18802920196E27928000092012270
:1068800001F0DAFEE0703B68002B20D0FFF7ACFF90
:10689000194D287800281AD0184B1978FFF778FE80
:1068A000002814D02B78E67808200793A78804F0F6
:1068B000D3FD011E09D0D0230370CA3B46708370FC
:1068C00087808671079804F077FE00232B701721CC
:1068D000A088FFF775FCA08801F034FCA08801F0C7
:1068E0000BFD09B0F0BD064B9DE7C0463409FF1F04
:1068F000B066FF1FC466FF1FA566FF1FA466FF1FCB
:106900001045FF1FF8B5070008000E0001F08AFED1
:10691000041E18D02620FFF78DFC051E00D1257817
:10692000062004F099FD041E0DD00021062204F07B
:10693000B3FDD0232370C23B21006770A370A680F3
:10694000E8B204F039FEF8BDF0B585B001930AABAA
:106950001B78070002930BAB1B7808000D00009218
:10696000039301F05FFE061E22D0102004F074FD98
:10697000041E1DD01022002104F08EFD2620FFF7FA
:1069800059FC002800D13078D0232370C13BA3707C
:10699000009B21002372019B67706372029BA5809C
:1069A000A372039BC0B2E3720C9BE36004F004FE8D
:1069B00005B0F0BDF7B50D00019001F033FE071EE4
:1069C00020D00E2004F048FD041E1BD02620FFF727
:1069D00031FC061E00D13E78D0232380C53B062221
:1069E000A370F91DE01C04F07FFD019B2A00638168
:1069F0000123DD401A401D40210022736573F0B26F
:106A000004F0DAFDF7BD0000F0B585B0029010008B
:106A10000D0017000A9E039301F004FE041E31D0FE
:106A2000029B002B2ED1039B02795B0724D51223F6
:106A300013430422002E08D10B99002905D10C998B
:106A4000002902D10D9900291AD01A430D9B2271F9
:106A5000002B00D0C9E0002E00D1CFE0002D00D0E7
:106A6000CCE0606A002801D004F0AEFE1C213000AA
:106A700004F07AFD606205E002239A430E33D7E703
:106A800093432371654BBA00D458002C00D1AAE07F
:106A9000002E10D0236A002B03D11C2004F05CFDD3
:106AA00020625E4BBA00D358186A002803D01C221B
:106AB000310004F019FD0C9B002B12D0574CBB0089
:106AC0001D596B6A002B03D1162004F045FD686246
:106AD000BB00E358586A002803D016220C9904F032
:106AE00003FD0D9B002B11D04C4DBC006659B36AC1
:106AF000002B03D1142004F02FFDB0622B59986AAB
:106B0000002803D014220D9904F0EEFC380001F0A7
:106B100089FD051E67D0414BBA00D358002B62D0C7
:106B20001A6A3420002A00D11C389A6A002A01D03F
:106B3000143080B20B9A002A01D01C3080B25B6AFC
:106B4000002B01D0163080B204F086FC041E4AD01F
:106B50001822002104F0A0FC2620FFF76BFB019017
:106B6000002801D12B780193D0232370029B2000B1
:106B700063700A23294EA370039BBD00A371AB5918
:106B8000A780196A1830002905D01C22A06004F0E3
:106B9000ABFC200034307359996A002907D00300F8
:106BA00014221433E060029304F09EFC02980B9BC5
:106BB000002B08D003001C221C330B992061029388
:106BC00004F092FC02987359596A002903D01622E6
:106BD000606104F089FC6B462100187904F0ECFC3C
:106BE0003800FFF7E3FC05B0F0BD10220D9B0D99B6
:106BF0001B69A018236204F077FC2CE70B9B002B89
:106C000000D13FE7012D00D03CE7606A002801D0A9
:106C100004F0DAFD1C210B982AE7C046AC66FF1F82
:106C200010B5044C2068002803D004F0CDFD0023EB
:106C3000236010BDA066FF1F0B4B07B51A68002A22
:106C400001D100200EBD6946531C01201278073186
:106C5000FFF772FC0028F4D00278012310001840DE
:106C60001A42EED0EEE7C046BC66FF1FF0B51F4FDC
:106C700001203B6887B0002B25D09B78059300F05E
:106C8000B3FB002821D00A20FFF7D4FA04000B2020
:106C9000FFF7D0FA164B05001E78731E9E413B6825
:106CA000F6B2191DD878FFF757FB3B682900DA7A4E
:106CB000043303929A7901930292009033002000EA
:106CC000059A04F049FE07B0F0BDFFF7B5FF0028B4
:106CD00005D00620FFF7AEFA04000720D8E7082009
:106CE000FFF7A8FA04000920D2E7C046A066FF1FFC
:106CF0009C66FF1F70B50A4E040033780D00FF2B11
:106D00000DD0042004F0A8FB011E08D0D02303708E
:106D1000CE3B45708370C470307804F04DFC70BD7C
:106D20002045FF1F70B5040006200D0004F094FB01
:106D3000011E0AD0D0230370CD3B8370054B4470F5
:106D40001B688580187804F037FC002C01D0FFF711
:106D500067FF70BDA066FF1FF8B5264F06003B68B1
:106D60000D001124002B05D10522234B1B78134263
:106D700002D112242000F8BD204A10241268002AF3
:106D8000F8D01278002AF5D0DB0719D52B789A1E97
:106D9000012A1AD80C2004F0DFFB132438600028E5
:106DA000E8D000230A22437029000670023004F064
:106DB0009BFBFFF75BFF041E0AD0FFF731FFD9E70B
:106DC00000F012FB0028E1D1E4E7002BE2D0D0E78D
:106DD0000B4B1B78032BCDD11D20FFF72BFA094B52
:106DE00018800028C6D0084B04211878074A04F000
:106DF00003FBBFE7A066FF1F9D66FF1FBC66FF1F6A
:106E00009C66FF1F9A66FF1FC866FF1F60EA0000AE
:106E1000F7B50193194B14001A78052306000F00EB
:106E200012201A4221D0012920D1154B1D68002DB6
:106E30001BD002201F2C18D8002C02D0019B002B45
:106E400013D0104B1F221E706E1C0021300004F066
:106E500023FB01992200300004F046FB31002000A2
:106E60002C70002F06D004F077FAFEBD064B1220DE
:106E70001D68DCE704F0D0FBF7E7C0469D66FF1F06
:106E8000BC66FF1F2045FF1FB866FF1FF8B50F4EF9
:106E900012243368002B17D01B780F3C834213D188
:106EA00000250B4F0221387804F036FA094B0421F3
:106EB00038781D8004F030FA074B28001D803368B5
:106EC0005C7004F001FB04002000F8BDA066FF1F09
:106ED000C866FF1FB466FF1F9A66FF1F70B50128C2
:106EE00023D11B4C2388002B03D01A4A1578002D80
:106EF00007D0194B1B68002B02D01878FFF7C6FF8C
:106F000070BD3B2B02D93C3B2380F9E7134E022195
:106F1000307804F001FAFA222388920002215A43C1
:106F2000307804F031FD2580EAE70B4B1B68002B1D
:106F3000E6D00B4B1B785B07E2D5084B0221187893
:106F400004F0EAF90022024B1A80FFF769FED7E746
:106F5000B466FF1F9866FF1FA066FF1FC866FF1F6D
:106F60009D66FF1FF8B51E4D2868002803D004F069
:106F70002BFC00232B601B4E3068002803D004F04C
:106F800023FC00233360184F05243B781800204071
:106F9000234221D0154800F02BFA3B78234213D02E
:106FA000202004F0D9FA2860002813D020220021E4
:106FB00004F072FA202004F0CFFA041E306005D0ED
:106FC0002022002104F068FA002004E0286804F080
:106FD000FBFB2C601320F8BD00F00AFAF4E7C04672
:106FE000BC66FF1FB866FF1F9D66FF1F1445FF1F8D
:106FF00010B50A4C23681A1E0ED0002808D10130A3
:10700000587004F061FA002805D02368002B02D0E4
:107010000021FFF787FE0122100010BDA066FF1FB0
:10702000F7B5274E050033680191181E21D05C7812
:10703000244F012C30D1FFF7FFFD002825D0200080
:10704000FFF7F8F80400412814D91F4B02211878E3
:107050001E4A04F0D1F91E4B3C3C1C8002223368CE
:107060005A703B78002B14D128000199FFF75AFE83
:107070000120FEBDFA2292004243002AEED0124BBC
:107080000221187804F080FCE8E7FFF7D3F802004B
:10709000F3E700233B70EBE73B78002BE8D10320BC
:1070A00004F0DAF9011E08D0D0230370CC3B457000
:1070B00083703368187804F07FFAFFF7B1FDD7E7E3
:1070C000A066FF1F9866FF1FC866FF1F60EA0000EA
:1070D000B466FF1F10B51749838802008B4220D089
:1070E00011D815498B4217D0144900205B1899B26A
:1070F000012907D8926811785A425341D8B2FFF754
:10710000F9FD012010BD0E4A00209B1807229BB2FA
:107110009A424041C0B2F5E783681878FFF768FFEC
:10712000F0E7836899785A78090218781143FFF7D5
:1071300077FFE7E70A20000006200000F8DFFFFFE6
:10714000AFDFFFFF014B18707047C0462145FF1F9E
:1071500010B5064C207001F041FA207804F0CCF80C
:107160000521207800F062FD10BDC046C866FF1FF3
:107170000BB273B50D00002B00DBC4E0884B187810
:1071800004F0E2FB041E0ED00378912B0FD0A22B4B
:1071900000D1A1E0834B1878FF2852D0210004F0E1
:1071A0000BFA00284DD180200002684076BD43785C
:1071B0000F2B76D013D8052B70D00E2BEAD18088F8
:1071C000794B98422BD8794B98421BD8784B9842F0
:1071D000E0D1A3681878591CFFF774F838E03E2B0B
:1071E000D8D18378032B74D06CD8012B6ED0022BAE
:1071F000D0D1704B1B68002B23D05B68002B20D0B4
:1072000098471EE06C4BC0180C28C3D804F0D4FA81
:107210001DC2C2150BC20B0B0B3223C23C00674BC5
:10722000C0180728B6D8664B1B68002B09D01B680E
:10723000002B06D0200098470AE0A3681878FFF7D3
:10724000C7F8200004F088FAADE7A068FFF762F8FD
:1072500000289FD0F5E7A3681B78002BF1D0554B91
:107260001B68002BEDD01B68002BEAD0210055488D
:107270009847EDE74F4B1B68002BE2D01B68002BB3
:10728000DFD021005048F3E7504B1B68002BD8D0CB
:107290005B68002BD5D021004348E9E7FFF7EAF906
:1072A000CFE780884A4B984203D04A4B984200D09F
:1072B00070E7464B1B68002BC3D05B68002BC0D027
:1072C0002100D5E7153B012BBBD963E7FFF798FAFF
:1072D000B7E7FFF77DFAB4E73F4B1B78042B07D1E4
:1072E00000236A4613800179408800F0C5FCA8E7B6
:1072F000364B1B68002BA4D05B68002BA1D001008B
:10730000364898479DE7012421420AD0294B1B6843
:10731000002B04D05B68002B01D00020984701208F
:1073200043E78B070AD5264B1B68002B04D05B680C
:10733000002B01D020009847022036E704212800C6
:1073400008400D4200D131E7254E3388002B21D073
:10735000013B9BB23380002B1AD1FFF7DBF80028EA
:107360000AD0204B1C70164B1B68002B04D05B68A6
:10737000002B01D020009847FFF7C6F8694601F0BE
:1073800001FD6846FEF7FEFF1D20FEF753FF30802B
:1073900004200AE7024B187803F0BEFFF8E7C04666
:1073A000C866FF1F2145FF1F0E20000001200000BE
:1073B00009100000C066FF1FFEDFFFFFAFDFFFFF09
:1073C000C466FF1F0C2000000B200000A866FF1FF2
:1073D0000D200000132000009D66FF1FFFFF00002E
:1073E0009A66FF1F9866FF1F10B501F09BF910BD4C
:1073F000014B18607047C046C466FF1F0B88002011
:10740000162B01D817230420014A13807047C04669
:107410007266FF1F00207047074A030011888142EF
:1074200007D091880020994202D1013080001018C5
:1074300070470020FAE7C046D066FF1FF0B58F788E
:1074400006000D00C7B01E2F15D1FFF7E5FF051E82
:1074500003D10024200047B0F0BD00223B003100E2
:10746000C078009200F0B2FB0400A81C00F0D3FB2F
:10747000FF23EB70EEE7264B062403931B78FF2BCC
:10748000E8D0182FE6D87B08224A013BDB000292A5
:107490009A589446002ADDD0029AD3185B68002BD4
:1074A000D8D00878002802D14B78012B02D10624CD
:1074B000122FCFD107AFAB88697800976446AA68CE
:1074C000A047041EC6D1AB78029A5B08013BDB00E3
:1074D000D318390030005B689847041E0BD1AB7895
:1074E000042BB6D0039A310010782200009700F0E8
:1074F0006DFB0400AEE76A78002AABD1AA7805A933
:107500003B88087130000A704B80FEF747FBA0E70C
:107510002445FF1FA4BB00111D4B37B50500984241
:107520000BD000290AD1FFF777FF002805D11948B1
:10753000FFF772FF002800D0058037BD01291AD15E
:10754000FFF76AFF041EF8D001235B420380A37893
:10755000FF2BF2D0FE2B07D00023E07814220093FB
:1075600029001E3300F032FBA01C00F054FB012365
:107570005B426380E1E70229DFD1013901F0BEF807
:107580000028DAD12800FFF747FF041EDFD1D4E737
:10759000FEFF0000FFFF0000022210B5074B524221
:1075A0001A80074801325A809A80DA8000F07EFA09
:1075B000044801F025F8002010BDC046D066FF1F2A
:1075C0003D740011197500110388F7B50400002BF4
:1075D00002D102252800FEBD426802211378254809
:1075E0005268FEF7A5FD00282ED0234F01253A88CA
:1075F000002AEFD0802321885B0201259B1A994243
:10760000E8DC0C2003F0A8FF061E31D03B8822885E
:107610009C4600231800019561469DB2491989B224
:10762000AA421BD8002801D062443A8000233000CF
:10763000082208C0210003F057FF104A1368002BEE
:1076400013D100251660C5E76268022113780C4843
:107650005268FEF76DFD0028C7D1BAE760681D01CA
:107660004019418101330198D6E71A001B68E6E70B
:107670001325AFE712BC00112245FF1FCC66FF1F88
:1076800010BC0011014B18707047C0462445FF1F05
:1076900014230A0010B51A40194204D00122102107
:1076A00001F048F810BD4B06F9D401208843400092
:1076B000F8E710B514008B0604D50122102101F063
:1076C00039F810BD08230A001A40194202D14BB202
:1076D000002B0FDA102101F02DF8002808D023002C
:1076E000F9331B78002BECD0F8342378012BE8D148
:1076F0000020E6E703208907FAD4E2E7F0B51F008F
:10770000184B85B01C68019002910392002C27D180
:10771000200005B0F0BDA5683301ED186B89019A12
:10772000934211D3029A93420ED8002F04D10A9BA0
:10773000002B10D12C00EBE73B002978039A6868F6
:10774000FEF7F6FC0028F2D10136B6B2A388B342A8
:10775000E1D82468DAE7A3680A9A5B891380E9E72D
:107760000026F3E7CC66FF1F37B50C000A8849886E
:107770000123914217D3002A15D0651D23792A00D1
:1077800002210A48FEF7D4FC102300280BD02379ED
:107790006188208800242A000094FFF7AFFF0A23A5
:1077A000A04200D0230018003EBDC04612BC00110C
:1077B00013B50A0008884988012388420BD800289D
:1077C00009D00024137905320094FFF797FF0A23AC
:1077D000A04200D02300180016BD13B50A00088887
:1077E0004988012388420BD8002809D00024137946
:1077F00005320094FFF782FF0A23A04200D0230045
:10780000180016BDF0B58BB003904A8808880E00AA
:107810000123824255D3002853D00023012704AC12
:1078200023700022718813000092FFF767FF051E86
:107830003ED02078002835D12B78022B18D16770E4
:107840006A8983000130E31880005A806968022247
:10785000201803F049FE23780133DBB22370042B98
:1078600019D93B006889013080B2002BD9D01FE0C4
:1078700002236370122358436A89231804305A8004
:1078800069681022201803F02FFE23780133DBB241
:107890002370002BE5D10C4A6B899B185A42534147
:1078A000DBB2DFE76378012BE4D12B78022BC7D062
:1078B00022780A23002A04D021000398FEF798F9C1
:1078C000002318000BB0F0BD0100FFFF0F4BF0B517
:1078D00004001868002816D083685D89A54207D87F
:1078E0008288AE18B44203DA12019A18934201D189
:1078F0000068EFE71E005F891036A74204D1002917
:1079000000D00D801800F0BD3300EFE7CC66FF1FFC
:1079100070B505000C0008880021FFF7D7FF0300B1
:107920000120002B04D022002800197AFFF7C1FEA5
:1079300070BDF7B50C00002501902300F6331B78CD
:10794000AB4201D800200AE06B00E65A002130006B
:10795000E718FFF7BBFF002802D126800130FEBDEB
:10796000017A0198FFF794FE002802D03B8823801B
:10797000F5E70135EDB2E0E710B504000888002115
:10798000FFF7A4FF03000120002B03D02000197A89
:10799000FFF77EFE10BD0000054B1B68002B01D1D8
:1079A000180004E09A6852898242F6D1988870479C
:1079B000CC66FF1FF0B50E27002687B0039302ABFD
:1079C000FF183E8005001F4B40891400984207D0E5
:1079D0002B78013000976A6880B2FFF78FFE0600AF
:1079E00002212B7818486A68FEF7A2FB00280FD006
:1079F0006C892000FFF7D0FF002802D0013C041959
:107A0000A4B2039B002B00D01C80300007B0F0BD57
:107A100002212B780D486A68FEF78AFB0028E7D11F
:107A200002212B780A486A68FEF782FB002807D0FB
:107A3000002EDED03B88A342DBD17489013CDFE716
:107A40006C89DEE7FFFF000012BC001110BC0011C2
:107A50000EBC001110B50C00FFF7DEFC0300022085
:107A6000002B0AD0002C00D023609B781720FE2B1F
:107A700003D00138FF2B00D1002010BD73B50D00DD
:107A800001A904001600FFF7E5FF172805D0002E16
:107A900004D129002000FEF727F976BD012210212C
:107AA000200000F047FE0028F3D0F6E7014B1860F5
:107AB0007047C046DC66FF1F37B56B469D1D010051
:107AC00004000222280003F07FFC2B88B02B0ED18B
:107AD0002379122B09D12300FF339B78012B06D188
:107AE0000121608800F0E0F801E01B2BF8D037BDE1
:107AF00010B5054B0421187000F098F8FFF74CFD05
:107B0000FEF770FB10BDC046E066FF1F0020F0B519
:107B10000BB20F0087B0834234DA274B187803F09A
:107B200013FF051E2BD00378A02B25D103AE310007
:107B3000FEF7E4F8041E0BD1B378DB0724D51F4B06
:107B400006341B68002B03D0310068889847040076
:107B5000A868002801D003F017FC002C08D1184AAF
:107B6000039B1340174A934206D0B3781B2B03D0D4
:107B70000121688800F098F8280003F0EDFD8020CE
:107B80000002784007B0F0BD0F4B1B68002B10D0EF
:107B9000310068889847041EDAD07378002BD7D15B
:107BA000B27801A90A704B800C716888FDF7F6FF66
:107BB000CEE70624F1E7C046E066FF1FD866FF1F48
:107BC00000FFFF0000011200DC66FF1FF7B5019007
:107BD000822040000D0017001E0003F03DFC040051
:107BE0001320002C12D0B02320002370089BFC220D
:107BF0006770658026710830002B08D0190003F0EB
:107C000073FC2100019803F0D7FC0020FEBD089909
:107C100003F042FCF5E710B5041E06D00078FD28FD
:107C200003D803F0A9FCFF23237010BD0A1F93B2F1
:107C300010B504000220032B05D882400020024B1F
:107C4000D1529B189C7010BD0067FF1F0B8870B548
:107C5000043B04000D000220032B0BD8012120005F
:107C600000F04CFD03001420002B03D0290020005D
:107C700000F0DEFB70BD000007B51300034A009260
:107C80000A00012100F02CFC0EBDC046B57E00119B
:107C900007B5019203220092024B0A00122100F064
:107CA00049FC0EBD337F001107B56B4601AA118058
:107CB0000449D88008780633012802D1190003F05E
:107CC0005BFE07BDE166FF1F0C4B10B5187000236B
:107CD000FF210B4A1380138193819380094A5380BB
:107CE0001370517293819372D174D382137551774B
:107CF00003F052FE00F0FCF910BDC0461067FF1FF4
:107D00000067FF1FE266FF1FF0B58DB06B460020D5
:107D100003910C229B5E834200DBB0E05D4B187840
:107D200003F012FE051E00D1A4E00378902B00D0D2
:107D30009DE006AF01004688380000F013FA79682C
:107D40000400002900D19CE03B88052B6ED13B89C3
:107D5000032B1CD905AC200000F0A2F86288172A7A
:107D600061D83989131D994231D17968237804315A
:107D70000291D90738D5607800F08EF9071E06D039
:107D8000002303712378012B08D0132B23D0A8687C
:107D9000002800D178E003F0F7FA75E062880299D4
:107DA00009A800F0A6F80290380000F08BF909AAA3
:107DB0002378387A0192002231000092029A00F072
:107DC00012F9380000F064F9029B002BDFD030007C
:107DD00000F080F9DBE70378032BD8D162880299A1
:107DE00009A800F0D6F8DEE7122B13D1029909A8F2
:107DF00000F0B5F8021EEAD127498B88002BC6D0C7
:107E0000887909A92378019161780091310000F007
:107E1000EAF8BCE7002302AA93833000617809AA3C
:107E2000FFF72AFFB3E71D4B0993F6E7042B02D0B7
:107E30009A1F012AABD8184A043B9B00995A002983
:107E4000A5D0D218907831003A0000F0AEF80028A2
:107E50009DD13B88042B03D001213000FFF724FF84
:107E6000012C04D1A868002801D003F08DFA280065
:107E700003F072FC8020039B0002434018000DB009
:107E8000F0BD012800D182E701213000FFF70CFF8F
:107E9000EDE7C0461067FF1F0067FF1F01001700D6
:107EA0000B7803704B784370CB788A781B021343AE
:107EB000438070470A88030002700A88120A4270E1
:107EC0000A88012A06D14A8882704A88120AC2703A
:107ED0000420704702208242FBD14A8804309A7005
:107EE0004A88120ADA708A881A718A88120A5A71C4
:107EF000EFE710B50400012082420CD94B780A78D4
:107F00001B0213432380834206D1CB788A781B025D
:107F100013436380002010BD022BFBD1CB788A78FD
:107F20001B02134363804B790A791B021343A3801E
:107F3000F0E70B8803700B881B0A43704B88837033
:107F40004B881B0AC3708B8803718B881B0A437193
:107F5000CB888371CB881B0AC3710820704703004C
:107F60000120082A14D14A780878120202431A80A4
:107F7000CA788878120202435A804A790879120234
:107F800002439A80CA798879120202430020DA807B
:107F9000704710B504000120022A05D100204B785B
:107FA0000A781B021343238010BDF8B50600102089
:107FB0000F00150003F050FA04000120002C0ED031
:107FC000A0230C22290023806780201D002D07D0CC
:107FD00003F08AFA2100300003F0EEFA0020F8BD29
:107FE00003F05AFAF6E7F7B51E00009008AB14202C
:107FF00017001D78019103F02FFA041E12D0A2235E
:108000000370019B47704380099B057146710C22E8
:108010000830002B07D0190003F066FA2100009801
:1080200003F0CAFAF7BD099903F036FAF6E737B557
:10803000041E0FD04388002B0CD00025C1881323C9
:10804000007A172201950095FFF7CDFFFF23658089
:108050006372257037BD000010B50C4904004A88D2
:10806000002A09D08B89002B05D00020CB8A022260
:10807000834201D010BD012213000A204343002097
:108080004032C854C81842800472F3E7E266FF1F0A
:108090000023438003707047094B00211A0010B57C
:1080A0005C88002C06D01C79844203D10A234B4300
:1080B000D01810BD01310A330329F1D10020F8E7AF
:1080C000E266FF1F10B50400407A03F055FAFF2363
:1080D000637210BD7047043010B580B203F0FCFA33
:1080E000002803D00421494203F05EFB10BD0000CC
:1080F00070B50025104CA0682580A581A580A842F8
:1081000002D003F041F9A56000250C4C0C4B606DCA
:108110001D80230058331D70A84202D003F034F9AB
:10812000656500256068002801D003F02DF9013550
:1081300008340A2DF6D170BDA867FF1F4C67FF1FDA
:108140009C67FF1F70B5041E09D1054D2880A881CA
:10815000A880A868002802D003F016F9AC6070BDB2
:10816000A867FF1FF0B54B8885B0019300234360DB
:108170000A7905000F00022A00D07BE0CA88032A92
:1081800017D98B685E7819783602DC78D8790E4377
:1081900099781B7A24021B020C43034353495BBAB0
:1081A0000B80331D93421ED1042C04D0631F022B7D
:1081B0000ED9012015E0019A4D4B1201D35A002B24
:1081C00006D00198FFF7BEFF4A4A136901331361D5
:1081D0000421B8682E812C80494203F0E5FA6860DA
:1081E000002005B0F0BD434D042C06D0631F022BC8
:1081F0000FD9EB680133EB60DBE7019A3C4B1201CE
:10820000D35A002B05D00198FFF79CFF2B6901334F
:108210002B61374B30000293019B029A1B010193A3
:10822000002301998C468B52130063449C80039376
:108230009E81FFF750FF039B041E986016D0042117
:10824000B868494203F0B0FAFA880100043A200005
:1082500003F04AF90199029AFB888A5A043B9B1859
:10826000029A8B522B6801332B60A2E7AB69013372
:10827000AB619EE71E4B0293019B1E01029BF35ACA
:10828000002B2DD002998C19A068002828D0012A33
:1082900026D1FA889B189BB27352A189994217D3B1
:1082A0009B1AC018B96803F01FF9029BA289F35A00
:1082B000934200D07DE700222B81A3882B80A36806
:1082C0006B60029BF2520B4A53680133536070E7B4
:1082D000084A9368013393600198FFF733FF68E71A
:1082E000044A536901335361F6E7C0461267FF1F22
:1082F000A867FF1F1867FF1F70B5051E15D10B4C2F
:108300000B4B1880230058331870606D002802D082
:1083100003F03AF86565250050356068002801D003
:1083200003F032F80834AC42F7D170BD4C67FF1F40
:108330009C67FF1FF0B51700A12285B09200019342
:108340004243394B06001B680C009B18D933FF339E
:108350001D78FDF741FF0430854204DD3000FDF754
:108360003BFF0430C5B2BD4207D33A0000213000C4
:10837000019B03F069FA05B0F0BD2900380003F055
:108380007BF82300C6B250331E700393019B290073
:108390006365380003F0A8FACBB20293002B02D039
:1083A000039B01361E7000262300503303931B7875
:1083B000B34204D8606D002831D10020DBE7029A77
:1083C0002800002A04D0013B1000B34200D028004E
:1083D000F700E719387003F037F9786000280ED0FD
:1083E0003A78019903F080F8019A3B780136D31866
:1083F0000E4A0193D369F6B20133D361D4E7039BEC
:1084000018706065A74205D1084A1320D36A01336A
:10841000D362B0E7606802F0B7FF0834F2E702F019
:10842000B3FF00236365C8E73409FF1F1867FF1F08
:10843000F7B50D0007000421686803F0B5F92B8932
:10844000040003702B891B0A43702B8883702B88D0
:108450001B0AC3702E8902250436F6B2FB2E15D8EE
:108460001B4B9F4214D10C2002F0F6FF1135011E68
:108470000CD0902303708E3B0371043B4380154B5B
:108480008460C680187803F097F800252800FEBDA8
:108490005C237B43104AD3180093583301931B7815
:1084A000002B0FD10300320038000099FFF742FF84
:1084B000019B05001B78002BE8D13800009903F0E0
:1084C000FBF8E3E7054A0725536A01335362DDE70A
:1084D000FEFF00001067FF1F4C67FF1F1867FF1F9C
:1084E000F0B587B0009017200F0016000193FFF73A
:1084F000F2FD1325041E19D00C98031E02D0019919
:10850000201D9847030AE370052302AAA0700430D7
:10851000908127700098667003A993800494FFF7F8
:1085200087FF051E02D0200002F02EFF280007B0B2
:10853000F0BD0000F0B587B01F000CAB1B780391B5
:10854000059301210DAB06001C78049200F0D6F8CB
:108550001425002821D02000FFF77EFD0135041EE0
:108560001BD01149059B0A7803700132D2B2131E49
:10857000C68001D101231A000B7022713000049BC8
:1085800003990097FFF7ACFF051E09D123002100D6
:108590000648074A093303F0EFF8280007B0F0BD9A
:1085A000002363802370F8E71467FF1F2F800011FA
:1085B00030750000F8B505000E00064C064F236824
:1085C000002B02D03100280098470434BC42F6D179
:1085D000F8BDC046B867FF1FCC67FF1F0123064ADE
:1085E0005B425380002313715362044A136053604B
:1085F0009360D36013617047CC67FF1FB867FF1F9C
:108600000200002310B506499C000859002801D13A
:10861000625010BD0133052BF6D11320F9E7C04697
:10862000B867FF1F034A5388181A43425841404213
:1086300010407047CC67FF1FF0B585B002930AABBE
:108640001F780CAB1B88009008000E00019203936A
:10865000FFF7E8FF05001120002D1BD10E48FFF7A2
:10866000E1FF04001520002C14D006220B99A771FD
:10867000E01D02F039FF019B30002371029B2900AD
:108680006371009B66802370039B6562E381FFF743
:1086900091FF280005B0F0BDFFFF000010B5FFF707
:1086A000C1FF04000220002C12D060880121FFF7D6
:1086B00081FF606A002801D003F086F8282200219B
:1086C000200002F0E9FE012300205B42638020715C
:1086D00010BD000030B5074A074C558801001378DB
:1086E0000020A54204D05B1A59424B415842104029
:1086F00030BDC046CC67FF1FFFFF0000084A10B521
:1087000001230C00904208D0FFF78CFF031E04D019
:10871000037923405A1E9341DBB2180010BDC046B6
:10872000FEFF0000024B1879431E9841C0B270470B
:10873000CC67FF1F70B504000D001600FFF772FF35
:10874000002804D10D4B9C4200D0143070BD416A0A
:1087500003790520002907D012221A40102A02D1DD
:108760000520002EF2D10F20DB06EFD5897E0C20EC
:10877000A9428941494249420840E7E7FEFF00001B
:10878000030010B5002800D110BD0348034A4188FA
:108790009142F9D09847F7E7CC67FF1FFFFF000031
:1087A000002330B5C45CCD5C6C40D4540133102B35
:1087B000F8D130BD0F23002210B5C45C6400224301
:1087C000CA54C25CD209013BF7D210BD02000100BD
:1087D00010B52032103102F09FFF10BDF0B58BB004
:1087E0000390102005931700049102F0B5FE00904D
:1087F000102002F0B1FE009B13240190002B05D045
:1088000000280CD11324009802F0DEFF019B002BFE
:1088100002D0180002F0D8FF20000BB0F0BD1020ED
:1088200002F09AFE0600102002F096FE13240500C6
:10883000002E00D1AEE0002819D01022002102F055
:108840002BFE32002900039802F066FF041E0ED1B1
:1088500033787F2B51D830000099FFF7ABFF009B96
:108860001B787F2B53D801990098FFF7A3FF3000A6
:1088700002F0AAFF002D02D0280002F0A5FF002C74
:10888000C1D1102002F068FE0600102002F064FE44
:108890000290002E7CD0002878D03A000F322300BE
:1088A0000125121105D00F333B4015B25A425341F6
:1088B0001BB26A1E1201002B33D0049BD2B298184F
:1088C0000099029AFFF76CFF013D10220021300051
:1088D00002F0E2FDADB2049F2D017D19AF4242D0FE
:1088E000002C33D0300002F06FFF029B002B00D130
:1088F00089E7180002F068FF85E729003000FFF7DC
:1089000059FF28002549009AFFF74AFFA7E72900E9
:108910000098FFF74FFF28002049019AFFF740FF1A
:10892000A5E70F210F4004998A18D9B28F4208D9C0
:10893000D15C06A819540133102BF6D1029A019983
:10894000C0E7791A48424141C901F2E739003000D5
:1089500006AAFFF725FF3200039806A902F0DCFE05
:1089600010370400BAE7002CBCD13000029906AAE7
:10897000FFF716FF320006A9039802F0CDFE082289
:1089800004003100059802F0AFFDABE71324A9E71E
:108990001324AAE7002800D06EE733E718BC0011C3
:1089A000F0B58BB00F0016000225009000283FD0D4
:1089B000002A3DD00B1DDBB21800029302F0CCFD63
:1089C0001135041E34D0FDF747FD05003A0000992B
:1089D000201D02F099FFEBB20393E3702B0CDBB286
:1089E0002F0A00936370FFB22B0E2370A7700193C0
:1089F000FDF72CFD1022010006A802F085FF2100E2
:108A0000029A04AB06A8FFF7E9FE051E0DD1039BF1
:108A100008223370009B04A9B370019B7770F37038
:108A2000301D02F071FFFDF71DFD200002F0CCFEAD
:108A300028000BB0F0BDF0B58FB00D00149E039070
:108A400004920593002A03D1022420000FB0F0BD48
:108A5000002EF9D00398FFF7E5FD1424071EF4D08B
:108A60007278337812021A43B3781B041343F278F6
:108A700012061A43036A0192934201D30133E3D1F0
:108A8000002D03D03B7901249B07DED5082200216D
:108A900006A802F001FD059B13240433DBB2180085
:108AA000029302F059FD051ECFD0059A04990430B7
:108AB00002F02AFF04223100280002F025FF3900CD
:108AC000102210310AA802F01FFF2900029A06ABFB
:108AD0000AA8FFF783FE041E0FD1082206A908A8E2
:108AE00002F012FF0822311D08A802F02DFD012816
:108AF00007D101990398FDF7C9FC280002F064FE34
:108B0000A3E70124F9E7000070B51C4C05002368B9
:108B1000181E10D0002D14D11A78002A0CD1981CE0
:108B2000083202F0E1FC02F01FFE0135002808D1F6
:108B300023681D70012070BD0A331800082202F05E
:108B4000D3FC2368002BF5D0122002F085FC061E12
:108B50000DD0C1232168037045700231102202300C
:108B600002F0C2FC23683100587802F025FD20682D
:108B700002F02AFE00232360DCE7C046F467FF1FF3
:108B8000F8B504002020FDF755FB0D4EA700BB599A
:108B90000500002B0DD000280BD0D878FF2809D174
:108BA00008492A000C55F35907480333611802F0AD
:108BB000E3FDF8BD290002F02FFC0028F0D1F8E712
:108BC0001068FF1FF867FF1FD99D001170B5064D93
:108BD00084006359002B05D0D87802F0CDFCFF2229
:108BE0006359DA7070BDC0461068FF1F70B506008B
:108BF0008CB00C00150000213022684602F04CFCBD
:108C000031001022684602F07FFE1D202100032261
:108C1000684402F079FE6846FFF7D8FD2D21040074
:108C200003222800694402F06FFE20000CB070BDE2
:108C3000F0B50700160097B001931CAB1D783022E9
:108C40001EAB00910AA800211C7802F025FC10221E
:108C500039000AA802F058FE1022002102A802F0F2
:108C60001BFC0722310002A802F04EFE072202ABD5
:108C70009818631E9C41019902F046FE02AB9C735A
:108C80002B005A1E934102AAD3730021102206A87A
:108C900002F002FC06221D9907A802F035FE1A20F8
:108CA00002ABC01806221F9902F02EFE1022009976
:108CB0000EA802F029FE102202AB0EA908781C783B
:108CC000013A6040D2B2087001330131002AF5D177
:108CD0000AA8FFF77BFD102212A904000EA802F0DB
:108CE00003FC102206AB0EA908781D78013A6840F3
:108CF000D2B2087001330131002AF5D10AA8FFF77A
:108D000065FD044310222098E4B212A902F0FCFD94
:108D1000200017B0F0BD70B50E0014008CB001003B
:108D2000102268461D0002F0EFFD3100082204A861
:108D300002F0EAFD2100082206A802F0E5FD6846DF
:108D4000FFF744FD04001022280008A902F0DCFD12
:108D500020000CB070BDF8B506000D0000243719D6
:108D6000AC4200D3F8BD02F08FFD030A3B70631CD8
:108D7000DBB201379D4203D90234F054E4B2EEE78E
:108D80001C00EDE773B506000C000225002819D081
:108D9000002917D0032101A8FFF7DDFF6B469A7960
:108DA0003F231A40013313436A463000937101A9EF
:108DB0002200FFF71BFF051E04D10322E01C01A9BE
:108DC00002F092FB280076BD03785807DA08C00F3E
:108DD000D20080009B0710439B0F1843C0B270471E
:108DE00007230B40C908C9000B43037070470000FC
:108DF00070B50400FFF7EAFE134DA4006359002B81
:108E000021D0186A002801D002F0DEFC2B59986EA0
:108E1000002801D002F0D8FC2B59D86E002801D0D0
:108E200002F0D2FC2B59186F002801D002F0CCFCC4
:108E30002B59586F002801D002F0C6FC285902F0C7
:108E4000C3FC00232B5170BD1068FF1F0E4B800028
:108E5000C35870B50C00002B0FD09D68002D0CD0AE
:108E60002B78201D0B706B784B70A97CFFF7B8FF37
:108E70002B7E23726B69E36070BD102200212000FD
:108E800002F00AFBF8E7C0461068FF1F014B1860AC
:108E90007047C0460C68FF1F074A030080008258D5
:108EA00010B5002A06D0D088984203D1012901D1FB
:108EB000FFF79EFF10BDC0461068FF1FF0B5264E9D
:108EC00095B087000B93BB590500099112200A92B7
:108ED000002B31D0D888FFF7A5FB04001420002C0C
:108EE0002AD0280010A9FFF7B1FFBB591E781D6AD0
:108EF000002E23D00895FDF7EFFA07000020FDF7BC
:108F0000F1FA0790A379E61D069310AD0CA9089815
:108F100000F0E2FA0EA9280000F0D7FA0B9B0A999C
:108F20000493069B09980293079B0396019300976D
:108F30000EAB0CAAFFF77CFE15B0F0BDFDF7CCFA26
:108F400006903000FDF7CEFAE31DA779079310AB2A
:108F500006000893DAE7C0461068FF1F30B50C4CD6
:108F600085002A59030085B00120002A0ED0180080
:108F70006946FFF76BFF2B591A78D888054B002AF2
:108F800000D1054B6A46072100F0D9FB05B030BD82
:108F90001068FF1FCB940011D994001130B5094C13
:108FA0008500295985B010226846253102F09CFAC7
:108FB0002A591121044BD0886A4600F0C0FB05B045
:108FC00030BDC0461068FF1F7595001130B5094CC3
:108FD0008500295985B010226846353102F084FA9F
:108FE0002A591121044BD0886A4600F0A8FB05B02D
:108FF00030BDC0461068FF1FB3950011F7B54D4F47
:1090000086001020F4590D0002F0A6FAF3592062F0
:10901000186A132200286CD0033A29009C6802F0D9
:1090200063FAF3591A780192002A58D11E6A227DF8
:10903000317B944651400122019F114201D1674684
:109040001740217D914339432175377B4F40BC4602
:1090500060460027800701D44F08174001210220F5
:109060008F40227D82433A432275377B5740BC466E
:1090700060460027400701D497080F400420227D56
:10908000BF0082433A432275627D002794466046C2
:10909000727B42400A4201D167460F400121627D46
:1090A0008A433A436275777B5740BC466046002747
:1090B000800701D457080F400220627D7F00824361
:1090C00017436775767B00227E40760701D4BA0885
:1090D0000A400426617D9200B1430A4362756A78B2
:1090E000002A08D06278002A05D005220533DA77F5
:1090F00000221000FEBD04222979114205D1A17C75
:10910000114202D10533033AF1E7019A21782C7814
:10911000002A02D10A002100140018220429E8D8EC
:10912000042CE6D805206043034A05331218525C2C
:10913000DDE7C0461068FF1F28BC001110B50A000B
:109140001121024B00F0FBFA10BDC0460F96001132
:109150000B0030B587B001AD2B806B4604001100C9
:10916000981D082202F0C0F92A000B212000024BB2
:1091700000F0E5FA07B030BD3796001110B50A00CF
:109180001121024B00F0DBFA10BDC0468B96001196
:1091900013B50B0011006A4613706B4604000622DB
:1091A000581C02F0A1F96A4608212000014B00F08A
:1091B000C6FA13BDAB96001110B50A001121024B7F
:1091C00000F0BDFA10BDC046FB9600117FB505004A
:1091D0000B4BAA00D4580800002C0FD0666F237FD9
:1091E000E28821780396266F0296E66E0196A46EB9
:1091F0000094FDF709FC2800FFF7FAFD7FBDC0468B
:109200001068FF1F10B51721FFF7E0FF10BD000029
:1092100070B50A000D00064B0221040000F08FFA21
:10922000060029782000FFF7D1FF300070BDC0464E
:10923000DB95001170B586B000236A461370836811
:1092400004001D78681E0A2859D801A902F024FBE1
:10925000060633373B3F43474B4F5300180000F09F
:1092600042F9062312284BD000281BD16088FFF753
:10927000D9F90823002813D04279002A47D1264B78
:109280001A78072312070BD5244B1A680723002AE4
:1092900006D01668002E03D0290001AAB0470300AB
:1092A0006A4613706B461B786088002B2AD1FFF743
:1092B00067FC06B070BD180000F06CF9D4E7180028
:1092C00000F087F9D0E7180000F093F9CCE7180018
:1092D00000F0ADF9C8E7180000F0C3F9C4E71800C2
:1092E00000F0F6F9C0E7180000F0F6F9BCE7180046
:1092F00000F013FAB8E7180000F013FAB4E70723F8
:109300006A46137069466088FFF782FFD1E705233C
:10931000012AC5D1024BB8E79D66FF1F0868FF1FF1
:109320000C68FF1FF8B52C4F8600F35904000D00A0
:10933000002B40D0DA8882423DD15A78062A33D1B8
:109340001A78002A2ED0012099681A6A097D0142F4
:1093500006D0157B054203D007225A700120F8BDC4
:109360000220014204D0157B054201D00922F4E716
:109370000420014204D0127B024201D00B22ECE710
:10938000164B1B68002BE9D05B68002BE6D0200051
:109390009847BB5900215B78122BDFD12000FFF7E3
:1093A00015FFDBE70E4BECE7112A04D1002900D0B2
:1093B00032252900F2E7002D08D12000FFF732F90D
:1093C000002803D0102302791343037121002800E1
:1093D000FDF798FAC2E7C0461068FF1F0868FF1F34
:1093E0000C68FF1F70B50E4E8500AB590400002BB2
:1093F00013D01B78002B11D10A4B1B68002B04D013
:109400005B68002B01D02000984773595B78122BC2
:1094100003D100212000FFF7D9FE70BD024BECE71D
:109420001068FF1F0C68FF1F0868FF1F094B8000B2
:10943000C3581020002B0CD01A6A002A09D09B6850
:10944000002B06D0127A1B7E101C9A4200D9181CE1
:10945000C0B270471068FF1F70B503000D00140004
:109460000220002A30D000292ED013700B78081D5E
:1094700053704B789370FFF7A7FCE0700120022136
:109480002B7A23716B7B034063716A7B0A40134321
:10949000042263716E7B1640334363716E7BF60862
:1094A000F600334363712B7B0340A371287B01409B
:1094B00000200B43A371297B0A401343A3712A7B2D
:1094C000D208D2001343A37170BD10B50A00010089
:1094D0000120FFF7C1FF10BD10B50A0001000220F6
:1094E000FFF7BAFF10BD70B506000C000220002E79
:1094F00030D000292ED07378201D0B70B3784B70BC
:10950000F178FFF76DFC01223579257271794B10E6
:10951000080013409340104003438810104080001F
:10952000C9080343C9000B436373B1794B100800AA
:109530001340934010400343881002409200C90832
:109540001343C9000B4321202373FCF773FE8542AC
:1095500001D2122070BD2220257AFCF76BFE8542D5
:10956000F7D823781820042BF4D86378012BF1D88E
:109570000020EFE7030010B50220002909D0002BDE
:1095800007D00322481C0A7019000D3201F0ACFF0D
:10959000002010BD03000222080010B5002B06D0E9
:1095A000002904D00E32591C01F09EFF0022100049
:1095B00010BD030010B50220002909D0002B07D0F0
:1095C0000422481C0A7019000C3201F08DFF0020A3
:1095D00010BD10B5FFF7DEFF10BD0300022000290B
:1095E00006D0002B04D0052200200A701B784B7097
:1095F000704703000220002B08D0002906D05B78BA
:1096000000200B70013B082B00D918307047030075
:1096100010B50220002909D0002B07D00622481CD3
:109620000A7019000A3201F05FFF002010BD10B56A
:10963000FFF7B0FF10BD02000B00022010B500299B
:109640000ED0002A0CD0072119701188597011888A
:10965000090A997011180822D81C01F045FF002052
:1096600010BD03000A00022010B5002B0CD0002909
:109670000AD099785878090201431180901CD91CAE
:10968000082201F031FF002010BD030010B50220B8
:10969000002909D0002B07D00822481C0A701900A5
:1096A000921801F021FF002010BD02000B000220E3
:1096B00010B500290BD0002A09D0092119701178A2
:1096C00018185970511C062201F00EFF002010BD21
:1096D00010B5FFF75FFF10BD02000B00022010B5B0
:1096E000002A09D0002907D05178197011180622D4
:1096F000581C01F0F9FE002010BD030010B5022037
:10970000002909D0002B07D00A22481C0A70190032
:10971000063201F0E9FE002010BD10B5FFF73AFF58
:1097200010BD02000B00022010B5002A06D000294F
:1097300004D018005178FFF753FB002010BDF0B59E
:1097400085B017001E006A460623050008009181B7
:109750009380FEF7C0FC1324011E02900CD0380049
:10976000B047041E05D1280001A9FEF76FFA041EB8
:1097700002D0029801F008FE2800FFF701FA20004D
:1097800005B0F0BDF0B504008BB0019115000021CB
:10979000102202A801F080FE334EA700B85900281D
:1097A0003CD0C388A34239D10378002B36D142780C
:1097B000062A18D102000100553235310C3006ABB3
:1097C000FFF7A9FA002829D12000FFF72FFE020099
:1097D00006A902A801F088FE200002A902F09CF868
:1097E00001200BB0F0BD816E002917D00B8A112A21
:1097F00028D19D420ED101981231093A01F0A4FE00
:10980000012807D1BB5920009D6EFFF70FFE2900EC
:109810000200DEE732212000FFF7D8FC2000FEF72F
:1098200001FF061E1BD0416A002918D00B8AAB42EB
:1098300015D108220198123101F086FE01280ED1BF
:10984000716A0AE09D42E9D108220198123101F0C3
:109850007BFE0128E2D1BB59996E8A7EB9E72000D0
:1098600002F082F8BCE7C0461068FF1FF0B56B4DF0
:1098700087007E5985B0337802900393002B00D087
:1098800087E0B368346A01937078062817D1012203
:109890001B7D134202D0217B114218D102221342B8
:1098A00002D0217B114251D10422134203D0237BE9
:1098B000134200D08BE0019B5A7DEB5991E00738B1
:1098C0000428F8D801F0E8FF032E42678300B36E46
:1098D000002B03D11C2001F03FFEB066EB599C6EBB
:1098E000002C1CD010220021200001F0D5FD029890
:1098F000FFF79CFD01002000FFF72DFA01F0C4FFE7
:109900002082200008211230FFF725FA0298FFF785
:109910008DFDA076EB592100D888FFF70FFC0822B7
:10992000EB591CE0B36E002B05D01A00198AF088A1
:109930001232FFF70DFC0222019B197DEB591142F7
:109940003DD0207B10423AD0073208E0F488FCF783
:10995000DBFD01002000FFF711FC0A22EB595A70D1
:10996000029B9C002A595378073B042B11D8D088BE
:10997000FEF758FE00284ED0C3895A08D21828494D
:10998000029B0298CB542B5941180433254801F00F
:10999000F3FE05B0F0BDFCF79FFD030001208342FC
:1099A00001D100200393EB59DE88FCF79BFD03995E
:1099B00002003000FFF7ECFB019AEB59117D042205
:1099C00011420CD0217B114209D00B22C7E7F68847
:1099D000FCF73CFD01003000FFF7EEFB6BE7019A5E
:1099E000527D01210A4204D0607B084201D00C2242
:1099F000B5E702210A4204D0607B084201D00E2262
:109A0000ADE704210A4204D0627B0A4201D0102251
:109A1000A5E71222A3E7FA225200B0E71068FF1F61
:109A20001468FF1FE39D001110B5064B1A7804233C
:109A3000100018401A4200D00348FFF727FA002010
:109A400010BDC0469D66FF1F2845FF1F70B504006E
:109A5000FFF7D4FA051E43D12000FFF77FFA234E0B
:109A6000A400A0598268937CDB0708D50321036A10
:109A70001B790B40012B02D1017F0B430377431D60
:109A8000D97F8B1E022B0DD8022900D00121C0885E
:109A9000FCF790FF042133591A7F59700A431A7753
:109AA000280070BD01290CD102231022437000212F
:109AB0000C3001F0F1FC305910213530FFF74BF933
:109AC000EEE70529ECD10223D118437010220C30A7
:109AD00001F00AFD04233259117F0B431377EAE7A3
:109AE00008251828DCD1053DDAE7C0461068FF1FBD
:109AF000F0B58BB0059143887E4F9E00F459150058
:109B00000493002C15D1012902D000200BB0F0BD28
:109B1000101D57781678FFF757F9EB68320002935B
:109B20002B7A0499019300903B002000FCF70CFF76
:109B3000EBE7E388049A934201D00820E6E7237814
:109B4000012B00D1D4E0059B581E092800D9CFE095
:109B500001F0A2FE05CE0A29CC506C859AB22900EC
:109B60000498FFF773FFD1E7200029001022453049
:109B700001F0BAFCB9594B78042B02D1013B4B7070
:109B8000C3E70B000A00253335320C310498FFF788
:109B900095F90498FFF702FA0522431E9841BB5934
:109BA000C0005A70B2E7200029001022553001F0A1
:109BB0009BFC049B4F4C9D00295904980A0006AB5E
:109BC00055320C31FFF77AF929591022453106A890
:109BD00001F0BAFC012808D10498FFF7F7F90590C5
:109BE000002804D106222B595A7005988EE70823C5
:109BF0000593FAE763780C2B7AD1E36E002B03D13F
:109C00001C2001F0A9FCE066BB59D86E00286FD07B
:109C10001022290001F068FCBB590498DC6EFFF7A4
:109C200005FC0D22A076BB595A706EE7E06E002845
:109C30005ED063780D2B5BD12B8808220382A91C90
:109C4000123001F051FCBB599A68517D0222114239
:109C500026D0186A407B104222D00C32E4E76378A9
:109C60000E2B45D1236F002B03D1162001F074FC7D
:109C70002067BB59186F002803D01022290001F07B
:109C800033FC0F22BB59CFE763780F2B30D1206F05
:109C90000622691C103001F027FCBB599A68517DDF
:109CA0000422114203D0196A497B1142D5D1002107
:109CB0000498FFF78BFA28E7636F002B0DD0BB5990
:109CC000586F0028F3D01022290001F00DFC01226A
:109CD000BB5952425B6F1A61E9E7142001F03CFC6A
:109CE000BB5960675B6F002BE9D126E72978DFE776
:109CF00007200BE71068FF1F10B5064C207001F01D
:109D000013FB06212078FDF791FF0348FEF778FC4E
:109D100010BDC0462368FF1F998E001100200BB2B2
:109D200070B50D00834216DA264B187801F00CFE50
:109D3000041E0DD00378922B0ED0A02B37D0224BCF
:109D40001878FF283AD0210001F036FC002835D1E0
:109D500080200002684070BD43780E2B0BD03E2B54
:109D6000EDD18378052B12D0082BE8D1817980883A
:109D7000FFF7D8FA08E0154B82889A42DFD1836852
:109D80001878591CFEF7C0FE002817D1D7E7104BF2
:109D90001B785B0712D50F4B1B68002B0ED09B68FE
:109DA000002B0BD0C289811D80889847ECE7FFF714
:109DB00041FAA068002801D001F0E6FA200001F085
:109DC000CBFCC5E72368FF1F2145FF1F18200000BB
:109DD0009D66FF1F0C68FF1F10B50078FFF712FA91
:109DE00010BD10B50078FFF7FDFA10BD0C234343FA
:109DF000084A10B59B185A68002A03D0012901D1DE
:109E0000904710BD9B68002BFBD00029F9D19847E3
:109E1000F7E7C0464068FF1F01238340094A10B599
:109E2000946B1C439463506B98435063D46B200035
:109E30009843012901D120001843D063116B0B43D3
:109E4000136310BD00800040F0B500240127154BBE
:109E500085B0DA6B144E03921A6C0192DA64019B9E
:109E6000E3403B4217D0039DE5403D400295E5B2FB
:109E700002992800FFF7BAFF316A736A002908D0F7
:109E80003900002B01D0029979402800FFF7C4FF68
:109E900001E0002BF9D101340C36172CDFD105B0CD
:109EA000F0BDC046008000402468FF1F064B012122
:109EB0005A68C2400A4204D01B68C34018000840D8
:109EC00070471B6DF9E7C046008000400122064B39
:109ED0008240002903D0D9680A43DA607047D96804
:109EE0009143D960FAE7C0460038004030B50324FA
:109EF00044430F4BE25C1B199C785D7801232D1BBA
:109F00000135AB40013BA340A140DB430C001228CC
:109F100007D808499200521811681940214311606E
:109F200030BD054A11680B4023431360F8E7C04673
:109F30006FBC001108F0004014F00040C21F70B563
:109F4000D4B20623092C0BD80125084C95400029D2
:109F500008D00021FFF7CAFF23682B4323600023AA
:109F6000180070BD2368AB43F8E7C04600380040D6
:109F7000214BF0B51B185B78022B21D103244443FD
:109F80001E4A1F4EA35C12199478012215008540C9
:109F9000B76B013CE4B23D43A240B563194C1228B3
:109FA00015D89B0000290CD117495B1899680A4302
:109FB0009A600123205C154A834011680B431360AB
:109FC000F0BD11495B18996891439960F1E70E4B18
:109FD00000290DD159690A435A61225C1328E8D03F
:109FE0000123203A93400A49086803430B60E7E7DE
:109FF000596991435961F0E72468FF1F6FBC001154
:10A0000000800040B4BC001100F00040A0F000400F
:10A01000A4F00040F8B500241B4E1C4D1C4B1B5DEA
:10A02000012B1FD1194A9269E2401A420BD001223A
:10A03000B25693402200143AD2B2022A09D81549E6
:10A040004A6913434B61013402360C35172CE5D1B4
:10A05000F8BD0022B2560F499200521891680B4386
:10A060009360F0E7022BEED1E7B23800FFF71EFF56
:10A0700001235840C1B23800FFF77AFF3800FFF7DC
:10A0800015FF6877DFE7C04641BC00112468FF1F59
:10A090002568FF1F00F00040012202388240054B76
:10A0A000002903D059690A435A617047596991439D
:10A0B0005961FAE700380040F8B50E0001210F00A1
:10A0C0008740114A0400D368FD43BB43D360831E1D
:10A0D0008B4201D8FFF7E0FF00212000FFF72EFFA1
:10A0E0000A4A0B4B5168012E05D139431B195160A7
:10A0F0005E700020F8BD2940516002221C19627078
:10A100009A6915409D61F4E70038004000800040E6
:10A110002468FF1F012210B58240074B002906D09A
:10A1200019680A431A600121FFF7C6FF10BD1968BC
:10A1300091431960F7E7C046008000400C2370B5DA
:10A14000002543430A4A29009B181D70094B04004F
:10A150001B185D70FFF7B0FF0123A34006492800DC
:10A160000A681A430A6005490A689A430A6070BD82
:10A170004068FF1F2468FF1F34800040308000408B
:10A1800070B504000E00FF2813D003250540FFF72B
:10A19000D5FF084AA3089B009B183F22ED00AA4068
:10A1A000AE40196820009143314319600121FFF747
:10A1B0008DFE70BD18380040F8B50C244443134B95
:10A1C0000500E4186368002B03D1A3681220002B5C
:10A1D0001AD0022201270E4B00215B195A70280069
:10A1E0002770FFF769FF63681E1E08D0A3683E0052
:10A1F000002B04D02800FFF759FE4640F6B2280095
:10A200003100FFF709FE0020F8BDC0464068FF1F7F
:10A210002468FF1FF7B5C420FF222B4B800019587C
:10A22000002491437F3A0A431A508022274F52025A
:10A23000274E1A60274B1D5D002D21D0A31E012B38
:10A2400003D80121E0B2FFF727FF012D18D11F4BE2
:10A250009B69E3402B4213D0E3B218000193FFF750
:10A2600025FE01000198FFF755FFE3B2143B022BD6
:10A270001DD801217156184A8D405369AB43536173
:10A280003B7F002B0DD0E5B22800FFF795FF28009B
:10A29000FFF70CFE7B7F0100834202D02800FFF70E
:10A2A000A5FD01340C370236172CC3D1F7BD0121AF
:10A2B00000237156F3568D40074A9B009B189A68FD
:10A2C000AA439A60DCE7C04600E100E02468FF1F73
:10A2D00041BC00112568FF1F00F0004010B50121AE
:10A2E0000400FFF7E9FE0123044A002011194B7016
:10A2F000A34091690B43936110BDC0462468FF1FC2
:10A3000070B50E0015000400FFF718FF0C2363431F
:10A31000094A20009B189D605E60FFF74DFFF02109
:10A32000064B074A8900051E5A5002D02000FFF74D
:10A3300005FF280070BDC0464068FF1F0000FF1FDA
:10A34000499E001170B5134D07202C78002C1FD1A9
:10A35000982221005200280001F066FA0123C4204F
:10A36000FF222B700C4B80001C635C630B4B1C604A
:10A370005C600B4B195891437F3A0A431A50802274
:10A3800052021A600D20074A074901F0A5FA200081
:10A3900070BDC0462468FF1F00800040A0F0004050
:10A3A00000E100E015A2001115A00011030010B596
:10A3B0000620072B09D8054A137000F0EDFFD721BE
:10A3C0000020034B034A89005A5010BD5045FF1F1F
:10A3D0000000FF1F151BFF1F70B51D0002240C2974
:10A3E00010D8094ACA40D2070CD5FBF72FFF041E2C
:10A3F00008D1059A04992800FBF744FFFCF7B2FD49
:10A40000FFF712FB200070BD1210000030B50D7870
:10A4100002232C009C43184201D02B431C0008252A
:10A420002300AB43284201D02B00234320241D00EE
:10A43000A543204201D01C4325002A230D70184259
:10A4400004D011781E3B0B43137030BD0028FCD1A3
:10A450000C2113788B43F7E7F8B51D0006AB1B887A
:10A46000140007AA0E000B201778002B27D10A78BA
:10A47000022A49D14A68507811780002244A0843D8
:10A480008018042840D801F007FA03121D1B23008E
:10A49000F06801F0B9F9021CC0B2B84200D93A1C08
:10A4A000D2B22000F1682A8001F01EF806E00222F4
:10A4B000F3681B882A8023701B0A63700020F8BD94
:10A4C0000622EEE701232B80F3681B782370F5E763
:10A4D000F368002B16D008222A801A8822701A8866
:10A4E000120A62705A88A2705A88120AE2709A8818
:10A4F00022719A88120A6271DA88A271DB881B0ABB
:10A50000E371DBE72B80D9E701202B80D7E7C0463A
:10A5100000D6FFFFF7B516000A781D0008AB1F88AC
:10A520000C000123022A18D14A68507811780002E1
:10A530002B4A0843801803280FD801F0ADF90225F3
:10A540004439E06801F060F9C0B20723B84204D38F
:10A550007B190193152B02DD0D231800FEBDE06869
:10A560002A003100C01900F0BFFF6B4600209B8815
:10A57000E268D0541B4B1B68834203D01B688342A4
:10A5800000D098470023E8E70B23002FE5D1022DE8
:10A59000E2D1737832781B021343E2681380114BC7
:10A5A0001B68002BEED01B68002BEBD00120E8E7E6
:10A5B0000B23002FD1D1062DCED12A003100E06827
:10A5C00000F092FFDEE70B23002FC6D1012DC3D18F
:10A5D00032787533012AC0D8E3681A70D2E7C046D2
:10A5E00000D6FFFF306AFF1F70B50C00150007286A
:10A5F00037D801F051F9041436361B36242E1820B2
:10A6000015290BD8184E16220021300000F044FF07
:10A6100022002900300000F067FF002070BD1820E4
:10A620000229FBD11288114B1A80F6E7182008295D
:10A63000F4D10A000E48290000F0C6FEEDE718200C
:10A640000129EBD10B4B10780B49DA69FFF7DEFEDD
:10A65000E3E718200129E1D1064B10780749DA6BAE
:10A66000F4E70220DAE7C046186AFF1FCE45FF1F55
:10A67000C445FF1F5445FF1F7C45FF1F9C45FF1F1E
:10A68000030010B50020DB0704D50721024A034868
:10A6900000F08CF810BDC046CCBC00115445FF1F23
:10A6A000054A03001068002803D082889A4201D12D
:10A6B000806870470068F6E7346CFF1F0A88030063
:10A6C00008009A4204D08A8804309A4200D00020C0
:10A6D00070470000F8B5F82200230D4F0D4E796841
:10A6E000050042433370994200D07B600A4C002140
:10A6F000200000F0D1FE00231A007C60AB4202D1A2
:10A7000000203370F8BD01332280DBB2F834F5E766
:10A71000346DFF1F306DFF1F386CFF1F73B56B4624
:10A7200001900600684615001980FCF74DFF041ED5
:10A7300011D1002D0FD07689002E11D00C2000F001
:10A740000BFF00280ED0084A0460136886808560DD
:10A75000002B02D11060200076BD1A001B68F7E7BD
:10A760000224F8E71324F6E7346CFF1F01210022CE
:10A770000A4B10B549420A4C198099809A719A7017
:10A78000084B2070012019805A60FFF7A3FF207842
:10A79000FCF778FF0448FDF733FF10BD386AFF1F50
:10A7A0003C6DFF1F346DFF1F59A80011022310B527
:10A7B000002802D0FFF7B2FF0300180010BD000010
:10A7C000030010B50020DB0704D50421024A03482A
:10A7D000FFF7A4FF10BDC046E0BC0011D445FF1F29
:10A7E000F0B50E2687B003930CAB1F8802ABF618AA
:10A7F0000500080031000292FDF768F8040001200E
:10A80000002C0FD03088FFF74BFF03000E20002BE9
:10A8100008D05E68002E05D021002800039B029A14
:10A820000097B04707B0F0BD0A4B10B5984207D16A
:10A830000122002352420A808B708A808B7110BDE6
:10A84000FFF73CFF0028FAD001235B42038000237E
:10A850008370F4E7FFFF0000F8B5050001290AD175
:10A86000134E00243388F827AB4219D02800114931
:10A87000FFF7DAFF06E0022904D10139FDF73EFFB8
:10A880000028EDD0F8BD3B0063437268D018D35A5E
:10A89000002B09D03A00002100F0FEFD0134E4B2A3
:10A8A000054B1B78A342EED801235B423380DDE7E2
:10A8B000346DFF1F386AFF1F306DFF1F10B5FFF7A3
:10A8C000FDFE03000020834200D0987810BD0000F8
:10A8D000F0B589B01C000EAB80CB03901E8810AB86
:10A8E0001B78049202930B7A0D00DB0616D42B78AA
:10A8F0000593022B24D00498FFF7D2FE002812D033
:10A9000003689C46002B0ED0029B22000193290075
:10A910003B00644603980096A04705E00498FFF7C3
:10A92000BFFE002802D10E2009B0F0BD8368002BC5
:10A93000F9D00A222900039898470028D7D0F3E7D6
:10A940006B6858781A786B4B000210439842D2D843
:10A95000043B984210D2684B984242D015D8674BBE
:10A96000C0180128C7D80B20002EDDD1EB681A785B
:10A9700059683A80200028E0614BC018032800D9AC
:10A9800079E000F089FF846A789E5E4B9842B2D1EC
:10A990000B20002EC8D101233B80EB6831001B78CF
:10A9A00023706889013080B2FCF790FF3A88031E5B
:10A9B0000ED0017802328A183A8042896270428948
:10A9C000120AA27059680278E01C00F08DFD06E0C2
:10A9D00004323A8031000422601C00F05DFD00204A
:10A9E000A2E70B20002E9FD1EB6807A91E88042345
:10A9F0003B80330A300026706370FCF767FF051E4A
:10AA000028D004AB9A890E2304A95B183E49C66876
:10AA1000FCF7D0FF00280BD12B783C486A680599D9
:10AA2000FBF786FB002803D1012304AA5B42D381F4
:10AA30003278022A06D17168201D00F055FD3B884E
:10AA400002333B800E2304AA9B181B88A3701B0AA9
:10AA5000E370C4E704ABDE81F4E70B20002E00D0E6
:10AA600062E7E9680398FFF729FF02233B80207023
:10AA7000000A6070B3E70B20002E00D054E70222DA
:10AA8000EB681B883A8023701B0A6370A7E7E868AD
:10AA900000F0BAFEC2B203000720B24200D243E780
:10AAA0000DD00299DBB27118994202DB921BD3B22E
:10AAB0000293029BE9681A003B8089195AE7002338
:10AAC000F6E70B20002E00D02EE70722EB683A8035
:10AAD0001A7822705A7862705A88A2705A88120ABC
:10AAE000E2701A792271DA886271DB881B0AA3711D
:10AAF00075E7C046042900000228000000D8FFFFC7
:10AB0000FFD6FFFF03280000FFFF000010BC00116C
:10AB1000F0B58DB06B460020089120229B5E8342E9
:10AB20003DDAA64B187800F00FFF071E32D00378ED
:10AB3000B02B2CD10079023816281FD800F054FD14
:10AB400017001E001E001E0031001E0096001E0091
:10AB50001D011E0052011E0073011E00CD011E00CA
:10AB600050021E001E001E008E021E00E302944BC7
:10AB700094491B8878880B80FBF71AF83800FCF79B
:10AB80009BFF914B1B68002B01D038009847380081
:10AB900000F0E2FD8020089B0002434018000DB049
:10ABA000F0BDF6220021874800F076FC0BAA3B7B23
:10ABB0007989388900923A000D32FCF79FFD040034
:10ABC000804B1B78002C3FD146E0804B7888059362
:10ABD0007F4B4100CB5A0BAE073BDBB2328802936E
:10ABE000002301937B4B210006930093059BFFF705
:10ABF0006FFE744D002810D1069B3A8A1B889A423A
:10AC00000BD138000599123000F09EFC002804D0CA
:10AC10002B7862899B00EB185A80162306A81B1814
:10AC2000328820007989FCF7C5FE2B7804009A0051
:10AC3000AA1851880029C3D00133DBB22B70002839
:10AC400007D006A9C98A9180634A12889A42BCD863
:10AC500002E0012149429180002B04D059497888B3
:10AC6000FAF7DAFF8AE73E890A2479E000253E896F
:10AC7000574B06937B88069A5B009B5A033B9D4289
:10AC800002DB002DF0D05BE0162206A812183B7BF9
:10AC9000798900923A0030000D32FCF72FFD0590C3
:10ACA000002858D04689017A7888FCF7F1FC041E08
:10ACB00044D1464B78880793069B4100C95A454BBF
:10ACC0000439C9B206AAD28A06930291019400936C
:10ACD0000599079BFFF7FCFD041E2FD1069B394900
:10ACE0001A88931C002D26D14B807988384B490057
:10ACF000CB5A5119033B8B4220DD059B31485B89C0
:10AD000041190B71A91C0135C9B2EDB20591451964
:10AD10001B0A2B71059B2D490433181800F0E4FB26
:10AD20002C4B059A1B88D318DDB22C4B9E4205D0C4
:10AD30000136B6B29CE749889942D6D0002D0CD096
:10AD4000204C2800618800F0D7FB20702100788813
:10AD5000FAF772FF12E7059CF0E7002C00D183E7B9
:10AD60007B78142B00D109E716493B794E800B7094
:10AD70000C717888FAF712FF00E7162406ABE41886
:10AD800021003889FCF7A2FD011E00D1B7E17888C7
:10AD900022880F4C45002C5B0A4D013CE4B2029422
:10ADA00000240F4B01940095FFF792FD041E00D084
:10ADB00014E129007888FAF74FFFDFE63C6DFF1FAA
:10ADC000C044FF1F406AFF1F346AFF1F3A6BFF1F1A
:10ADD0007066FF1F306CFF1FBE44FF1FFFFF0000A7
:10ADE000426AFF1F162406ABE41821003889FCF7DD
:10ADF0006DFD011E00D182E178882288AE4C4500AD
:10AE00002C5BAE4D013CE4B202947C89AC4B0194C6
:10AE10000095FFF75DFD041E00D0DFE02900788873
:10AE2000FAF724FFAAE60025A44B1D803B00FE3361
:10AE30001B78A24A78880792AB4208D99E4B1288A9
:10AE40000693069943005B5A013B9A4203DB07993C
:10AE5000FAF716FF92E616246B00FB18059306AB73
:10AE6000E418059B21001889FCF730FD011E03D171
:10AE7000059B01241E8973E77888924B2288069CE3
:10AE8000099343001B5B904E013BDBB2029300230E
:10AE900000960193099BFFF71BFD041E02D0059B42
:10AEA0001E895DE77B88069A5B009B5A079A10888B
:10AEB00032881218934202DC1B1A013B33807F4C0C
:10AEC000023032880999001900F00EFB238832887D
:10AED00001359B182380EDB2A8E70BAA3B7B79894B
:10AEE000388900923A000D32FCF708FC00250590E5
:10AEF000059B002B04D10A24002D00D16EE060E0F8
:10AF0000059B7888197AFCF7C3FB0100041E63D106
:10AF1000694C6C4B788806940993069B4400E45A6C
:10AF2000694B063CE4B20BAE328807930294019160
:10AF300000930599099BFFF7CBFC041E4CD1079B9E
:10AF40005E491B881A1D002D30D14A80059B5B4C41
:10AF50005A8963191A716B1C9BB2E318120A1A7191
:10AF6000162306A832881B1879890598FCF722FD5C
:10AF7000FF21AA1C2E1D03350B00059092B2B6B21C
:10AF8000ADB2002803D006ABDB8AD9B21B0AA218E7
:10AF9000651911712B714C4D301D2A8849492018B3
:10AFA00000F0A2FA2B88F618B5B2A1E749889142C1
:10AFB00007D17A8806995200525AEB18053A9A42FC
:10AFC000C4DC3E4C2800618800F056FA2070210055
:10AFD0007888FAF75FFED1E5002DF2D13E89BFE611
:10AFE000162606ABF61831003889FCF76FFC3D00D9
:10AFF0000400FF3500282DD0037A9B060CD40022D4
:10B000007B893989788800923A000C32FFF7E8FB97
:10B01000041E10D03E8915E03088FFF741FB002860
:10B020001AD08368002B17D0210012227888984705
:10B03000041EE4D0EEE7AB78002B02D17888FAF753
:10B0400039FE0026AB78002B00D097E5002C00D10C
:10B0500094E585E60124DDE70E24DBE7162506AB43
:10B06000ED1829003889FCF731FC041E47D0037A1B
:10B070009B0611D4154A7B881188994203D0144845
:10B08000814207D11380134BF8261D780023D9B2D3
:10B09000A94221D30924A1E72888FFF701FB002852
:10B0A0002FD08368002B2CD021001222788898475B
:10B0B000041EDFD092E7C0467066FF1F406AFF1F84
:10B0C000426AFF1F3A6BFF1F306CFF1F346DFF1F7A
:10B0D000FFFF0000306DFF1F3100594354680133FA
:10B0E0006018615A0029D2D13C0008342100F822AE
:10B0F00000F0FAF921007888FAF7E4FD3EE5012432
:10B100006CE70E246AE71D4B1A887B889A4231D07F
:10B110007888FAF7E1FD31E5F82305985168434353
:10B12000CD18C95A00291FD03B7A012B0BD16C884E
:10B13000AB887888AA1D0094FFF752FB041E02D04A
:10B1400000233B722E88F8220021280000F0A4F989
:10B1500000232B80059B0133DBB20593084B059937
:10B160001B78064A8B42D7D801235B421380002C00
:10B17000CED0F5E5002634000596EFE7346DFF1FCD
:10B18000306DFF1F70B504000E001500FFF796FA32
:10B19000031E08D131000548FFF790FA0300112083
:10B1A000002B02D01C8000209D7070BDFFFF0000AE
:10B1B000F8B50B4F06003B780D001400FF2B0ED0A6
:10B1C0000A2000F049F9011E09D0B12303800023B1
:10B1D00046800371C5800481387800F0EDF9F8BD30
:10B1E0001546FF1FF7B50F0008A90600088809A932
:10B1F0000B240988002821D10234022B1ED1557856
:10B2000013782D021D432B008B4301937334002BC5
:10B2100014D1FB68300019000093FFF74FFB019C2D
:10B2200085420BD02A0030000099FFF7ABFF041EC7
:10B2300004D12A0030007989FFF7BAFF2000FEBD53
:10B24000F0B50E7885B003900AA805880120022E7B
:10B250000DD14C682778647824023C43054FBC42EA
:10B2600005D10398DBB201960095FFF7BBFF05B04F
:10B27000F0BDC0460229000010B504000C4800F0E3
:10B2800083FA0C48A16B00F07FFA0B48E16B00F0E9
:10B290007BFA0A48216C00F077FA094B09481968D3
:10B2A00000F072FA084B1B68002B00D09847FEE7AD
:10B2B000E2BA0011F8BA001107BB001116BB001169
:10B2C00004ED00E025BB0011406DFF1F002307B512
:10B2D00001A80193FFF7D0FF044A0548002110B5EB
:10B2E000121A00F0D9F8F8F765FBFEE7446DFF1F6E
:10B2F0001846FF1F0000000001B40248844601BC4C
:10B30000604700BF5D17000001B40248844601BCDD
:10B31000604700BF9DA9000001B40248844601BCFB
:10B32000604700BFB352010001B40248844601BC2B
:10B33000604700BFC926000001B40248844601BC32
:10B34000604700BFF539FF1F01B40248844601BCC5
:10B35000604700BF5125000001B40248844601BC8B
:10B36000604700BF4D1F000001B40248844601BC85
:10B37000604700BFB14E000001B40248844601BCE2
:10B38000604700BFC9A9000001B40248844601BC5F
:10B39000604700BFD949010001B40248844601BC9E
:10B3A000604700BF151BFF1F01B40248844601BC63
:10B3B000604700BFA134FF1F01B40248844601BCAE
:10B3C000604700BFADAE000001B40248844601BC36
:10B3D000604700BF810E000001B40248844601BCF2
:10B3E000604700BF3555000001B40248844601BCE7
:10B3F000604700BF456B010001B40248844601BCB0
:10B40000604700BF5952010001B40248844601BCA4
:10B41000604700BF8538FF1F01B40248844601BC65
:10B42000604700BF5147010001B40248844601BC97
:10B43000604700BF3939FF1F01B40248844601BC90
:10B44000604700BF8552010001B40248844601BC38
:10B45000604700BFC56D010001B40248844601BCCD
:10B46000604700BF1D4D010001B40248844601BC85
:10B47000604700BF3D18000001B40248844601BC8B
:10B48000604700BF090E000001B40248844601BCB9
:10B49000604700BF4135FF1F01B40248844601BC2C
:10B4A000604700BF154D010001B40248844601BC4D
:10B4B000604700BF056A000001B40248844601BC31
:10B4C000604700BF813AFF1F01B40248844601BCB7
:10B4D000604700BF691F000001B40248844601BCF8
:10B4E000604700BFC94A010001B40248844601BC5C
:10B4F000604700BFE94C010001B40248844601BC2A
:10B50000604700BF350E000001B40248844601BC0C
:10B51000604700BF0189000001B40248844601BCB5
:10B52000604700BF156B010001B40248844601BCAE
:10B53000604700BF4550000001B40248844601BC8A
:10B54000604700BFB537FF1F01B40248844601BC05
:10B55000604700BFCD4C010001B40248844601BCE5
:10B56000604700BF3D4B010001B40248844601BC66
:10B57000604700BFF94C010001B40248844601BC99
:10B58000604700BF1147010001B40248844601BC76
:10B59000604700BF2D3BFF1F01B40248844601BC39
:10B5A000604700BF3136FF1F01B40248844601BC2A
:10B5B000604700BFC13AFF1F01B40248844601BC86
:10B5C000604700BF594F010001B40248844601BCE6
:10B5D000604700BFF30E000001B40248844601BC7E
:10B5E000604700BFB54C010001B40248844601BC6D
:10B5F000604700BFF93CFF1F01B40248844601BC0C
:10B60000604700BFD1A5000001B40248844601BCD8
:10B61000604700BF055E000001B40248844601BCDB
:10B62000604700BF5522000001B40248844601BCB7
:10B63000604700BF6571010001B40248844601BC47
:10B64000604700BFA93BFF1F01B40248844601BC0C
:10B65000604700BF017F000001B40248844601BC7E
:10B66000604700BF9137FF1F01B40248844601BC08
:10B67000604700BFDD30FF1F01B40248844601BCB3
:10B68000604700BFDD66010001B40248844601BC8A
:10B69000604700BFA54F010001B40248844601BCC9
:10B6A000604700BF1D4B010001B40248844601BC45
:10B6B000604700BF8132FF1F01B40248844601BCCD
:10B6C000604700BF7D18FF1F01B40248844601BCDB
:10B6D000604700BF2146010001B40248844601BC16
:10B6E000604700BFE928000001B40248844601BC5D
:10B6F000604700BF2526000001B40248844601BC13
:10B70000604700BF2124000001B40248844601BC08
:10B71000604700BF6DBC000001B40248844601BC14
:10B72000604700BFE548000001B40248844601BC00
:10B73000604700BFEDA5000001B40248844601BC8B
:10B74000604700BF8D12000001B40248844601BC6E
:10B75000604700BFC95C010001B40248844601BCD7
:10B76000604700BF434D010001B40248844601BC5C
:10B77000604700BFD91B000001B40248844601BCE9
:10B78000604700BFA946010001B40248844601BCDD
:10B79000604700BFE53A010001B40248844601BC9D
:10B7A000604700BFE134FF1F01B40248844601BC7A
:10B7B000604700BF5549010001B40248844601BCFE
:10B7C000604700BFD13CFF1F01B40248844601BC62
:10B7D000604700BF014C010001B40248844601BC2F
:10B7E000604700BF75A9000001B40248844601BC4F
:10B7F000604700BF9130FF1F01B40248844601BC7E
:10B80000604700BF413AFF1F01B40248844601BCB3
:10B81000604700BFDD52010001B40248844601BC0C
:10B82000604700BF291C000001B40248844601BCE7
:10B83000604700BFB70E000001B40248844601BC57
:10B84000604700BFC51D000001B40248844601BC2A
:10B85000604700BF5118FF1F01B40248844601BC75
:10B86000604700BFD53BFF1F01B40248844601BCBE
:10B87000604700BF6932FF1F01B40248844601BC23
:10B88000604700BFC521000001B40248844601BCE6
:10B89000604700BF2951010001B40248844601BC41
:10B8A000604700BFE53CFF1F01B40248844601BC6D
:10B8B000604700BF0124000001B40248844601BC77
:10B8C000604700BF0D52010001B40248844601BC2C
:10B8D000604700BFC53F000001B40248844601BC78
:10B8E000604700BF0933FF1F01B40248844601BC12
:10B8F000604700BF090E000001B40248844601BC45
:10B90000604700BF093AFF1F01B40248844601BCEA
:10B91000604700BF4551010001B40248844601BCA4
:10B92000604700BF311B000001B40248844601BCDF
:10B93000604700BFED4A010001B40248844601BCE3
:10B94000604700BFC132FF1F01B40248844601BCFA
:10B95000604700BFF54E010001B40248844601BCB7
:10B96000604700BF851F000001B40248844601BC47
:10B97000604700BF091B000001B40248844601BCB7
:10B98000604700BFE117000001B40248844601BCD3
:10B99000604700BF8B52010001B40248844601BCDD
:08B9A000604700BF79180000A8
:10B9A800000201030203030304030502060207025F
:10B9B800080209000A030B030C020D000E030F0313
:10B9C800100311031303140315001600993D001109
:10B9D800CD3D00110000000002000000EAB900118E
:10B9E800192A0F180A000000F1590000FD24000070
:10B9F80041460100097D00111D9D00117171001162
:10BA08000D7B00111953001111AB00118D4F00115E
:10BA1800F93F00112941001100000000161600002E
:10BA28000200000034BA0011F4FFF3FFD2FC00005A
:10BA3800F541001100000000000000005475796114
:10BA48000042312E32003030303100676974687539
:10BA5800622E636F6D2F70767678004254483031CD
:10BA6800000000000200000080BA0011292A282ADC
:10BA7800272A262A252A242A0A180000E204000078
:10BA88007102000078EC00007440000010270000EC
:10BA980060F0000006640000204E00000000000076
:10BAA800010000001F501D00023CB40000011400FA
:10BAB800120000008102000030313233343536374D
:10BAC8003839414243444546005048592B3632588C
:10BAD80058504C555330353034005B4861726420FF
:10BAE8006661756C742068616E646C65725D0A00CD
:10BAF8004C522020203D203078253038780A0050DC
:10BB0800432020203D203078253038780A005053D3
:10BB18005220203D203078253038780A0049435398
:10BB280052203D203078253038780A001D57001102
:10BB38007157001100000000020000004CBB00110A
:10BB48006F2A6E2A1A18000001A0000000000000E9
:10BB58006410B71DC8206E3BAC30D9269041DC7606
:10BB6800F4516B6B5861B24D3C7105502083B8EDB0
:10BB780044930FF0E8A3D6D68CB361CBB0C2649BD4
:10BB8800D4D2D38678E20AA01CF2BDBDFB349B5FF9
:10BB9800800000800010000000000000735D0011AC
:10BBA800FD730011975D0011057800111B5E0011EF
:10BBB800DB770011915E0011B1770011E35E00118F
:10BBC800797900114B5F0011797900117D5F0011BF
:10BBD80033790011915E001169770011095F001136
:10BBE800117900110000000000000000EF5F001153
:10BBF800117900115160001115740011052A042AE9
:10BC0800012A002A022903280128002801180018FF
:10BC18000000000000000000000000000000008795
:10BC280001010201020101020102030304010301EF
:10BC3800010101010303020103000D000E001000C1
:10BC4800110013001401070108010A010B011C016E
:10BC58001D02040205020702080219021A021C0248
:10BC68001D03010302031700020100050400080771
:10BC7800000B0A001716001D1C0102010105040132
:10BC88000E0D011110011413011716011A190202E1
:10BC980001020B0A020E0D021110021413021716EC
:10BCA800030504030807030B0A030E0D0001020332
:10BCB80007090A0B0E0F101112141718191A1B1F57
:10BCC8002021220059A4001115A500110000000030
:10BCD8000200000016BC00110000000041B2001173
:0CBCE800000000000200000014BC00116D
:020000041FFFDC
:1000000000000000F53E0011F0B90011ECB900113C
:100010002463FF1F0000000000000000000000003B
:1000200000000000000000000000000000000000D0
:1000300000000000000000000000000000000000C0
:1000400000000000000000000000000000000000B0
:1000500000000000000000000000000000000000A0
:100060000000000000000000000000000000000090
:100070000000000000000000000000000000000080
:100080000000000000000000000000000000000070
:100090000000000000000000000000000000000060
:1000A0000000000000000000000000000000000050
:1000B0000000000000000000000000000000000040
:1000C0000000000000000000000000000000000030
:1000D0000000000000000000000000000000000020
:1000E0000000000000000000000000000000000010
:1000F0000000000000000000000000000000000000
:1001000000000000000000000000000000000000EF
:1001100000000000000000000000000000000000DF
:1001200000000000000000000000000000000000CF
:1001300000000000000000000000000000000000BF
:1001400000000000000000000000000000000000AF
:10015000000000000000000000000000000000009F
:10016000000000000000000000000000000000008F
:10017000000000000000000000000000000000007F
:10018000000000000000000000000000000000006F
:100190000535FF1F5533FF1FC16601000000000039
:1001A000000000000000000000000000000000004F
:1001B000000000000000000000000000000000003F
:1001C000000000000000000000000000000000002F
:1001D000000000000000000000000000000000001F
:1001E000000000000000000000000000000000000F
:1001F00000000000000000000000000000000000FF
:1002000000000000000000000000000000000000EE
:1002100000000000000000000000000000000000DE
:1002200000000000000000000000000000000000CE
:1002300000000000000000000000000000000000BE
:1002400000000000000000000000000000000000AE
:10025000000000000000000000000000000000009E
:10026000000000000000000000000000000000008E
:10027000000000000000000000000000000000007E
:10028000000000000000000000000000000000006E
:10029000000000000000000000000000000000005E
:1002A000000000000000000000000000000000004E
:1002B000000000000000000000000000000000003E
:1002C000000000000000000000000000000000002E
:1002D000000000000000000000000000000000001E
:1002E000000000000000000000000000000000000E
:1002F00000000000000000000000000000000000FE
:1003000000000000000000000000000000000000ED
:1003100000000000000000000000000000000000DD
:1003200000000000000000000000000000000000CD
:1003300000000000000000000000000000000000BD
:1003400000000000000000000000000000000000AD
:10035000000000000000000000000000000000009D
:10036000000000000000000000000000000000008D
:10037000CDB20011000000000000000000000000ED
:10038000000000000000000000000000000000006D
:10039000000000000000000000000000000000005D
:1003A000000000000000000000000000951AFF1F80
:1003B000000000000000000000000000000000003D
:1003C000000000000000000000000000000000002D
:1003D000000000000000000000000000000000001D
:1003E000000000000000000000000000000000000D
:1003F00000000000000000000000000000000000FD
:081838005071FF1F4118FF1F52
:10184000024981F3088802F023FC00005071FF1F59
:1018500010B502F025FB072804D0122808D0022872
:1018600008D010BD044A0420136B01331363F8E75A
:101870000220F6E71420F4E71867FF1FF8B5070009
:101880000C0026002500503630785135002804D150
:101890000300287058342370F8BD2978CA00481E08
:1018A0008141A3183800A25C5B68C9B2FFF7D0FF82
:1018B00000280DD12B78DA00A218013350602B706C
:1018C0003378044A013B3370136A01331362D8E75B
:1018D0000123DFE71867FF1F5C234343074910B567
:1018E000C9180B0058331B78012B05D1FFF7C6FF31
:1018F000034A936A0133936210BDC0464C67FF1FD1
:101900001867FF1F10B502F01BFC064A01211300E7
:1019100010CB4942D967044B136002F051FC200000
:1019200010BDC04600E100E01000100010B504003A
:1019300002F006FC024B1C6002F042FC10BDC046E7
:1019400000E100E010B5040002F0FAFB4021094A72
:10195000200013688B43136002F04AFB01F0B4FDD2
:101960000022054B01201A60044B04321A6002F079
:10197000CFFAFEE71CF00040C4F00040C0F0004089
:10198000431E5A425341A022F0B5D2015B4213409C
:10199000154D164A40019B182A18127E8BB00191F2
:1019A000002A1BD01A000832D46F0022E6B206AF1C
:1019B000E4B294420EDC2818C369002B08D00199C8
:1019C00002AA117106AA049202AA167303A89847E4
:1019D0000BB0F0BD1978B9540132EAE71A7D1A78D4
:1019E00006AB01261A70E6E7D869FF1F00400040E9
:1019F000F0B5254B04004001C25C85B0002A2BD015
:101A00001A18117E002927D0917E002924D011793F
:101A1000022921D11689D788D168F51BADB22A1CBD
:101A2000102D00D9102292B2BE4217D118180123EE
:101A300003710023C269C38003819A4206D06846BD
:101A4000032103730171029301A890470820002C21
:101A500000D0192001F034FC05B0F0BD013C654216
:101A60006C41A0256442ED012C40084D1B186419FF
:101A7000074D0633013A92B2AA42EDD01888461CAF
:101A80001E80085C2070F5E7D869FF1F0040004009
:101A9000FFFF00000F220E4B10B59868104002386F
:101AA0000A280BD802F01EF90D0A0B0A0A110A0ABD
:101AB0000A0A060002210020FFF762FF10BD012183
:101AC000F9E70020FFF794FFF8E7DB6FF6E7C04681
:101AD000004000400F220E4B10B5986810400238AD
:101AE0000A280BD802F0FEF80E0A0B0A0A120A0A9C
:101AF0000A0A060002210120FFF742FF10BD012162
:101B00000800F9E70120FFF773FFF7E7DB6FF5E760
:101B10000090004013B5334C2378072B3DD8324B4F
:101B20001A78324B002A39D18022196852020A43AE
:101B30001A60252001F084FF20232D4A11680B43F1
:101B4000802113606B460422C905086807331042E0
:101B500028D080210422C905C86810422ED08021D7
:101B60002020C905CA688243CA6014221A701A78F4
:101B7000002A2FD18021C905C86820320243CA60DB
:101B800014221A701A78002A28D11A4B1A7D22784A
:101B90005A601D221A705932DA6013BD1A6816494C
:101BA0000A40C5E7086802430A6014221A701A78CE
:101BB000002ACED01A78013AD2B2F7E7C8680243B9
:101BC000CA6014221A7019784A1ED2B21A700029FB
:101BD000F9D1C4E71A78013AD2B2C7E71A78013AC4
:101BE000D2B2CEE75045FF1F1846FF1F3CF0004021
:101BF0004845FF1F00200040FFFFFEFF564B70B519
:101C00001B68012B03D1554A936D0133936502F094
:101C1000AFF8534B534A1860534B544C1A6001238E
:101C2000534A1360534A13602378002B06D00622D0
:101C30005149524802F004FA00232370504A514B94
:101C400010681B78C1B2002B0ED14F4CC0B2237864
:101C50005BB2002B4FDB237824785BB264B21B04A9
:101C600024021B191B1813600B1C50294ED950233A
:101C7000464A47491078DBB2FF2202284BD1086858
:101C8000444C454D267890432A78964254D9227880
:101C900024782E78023B5D10A31B6B435201D31AAC
:101CA00010335B111843086002F0E2F8031F012BA8
:101CB00045D83A4B1B78002B06D0394B1B78002BAC
:101CC00002D0002002F04CFAA122364B9200997803
:101CD000354B4A431B689B18832292009B181B7844
:101CE000033B012B03D8AF20400002F029F9012269
:101CF0002E4BDA8270BD237824785BB264B2FF3356
:101D0000FF341B0424021B190138ABE7CAB2022AB4
:101D1000AED20223ACE70868254C264D26789043C6
:101D20002A78964208D9227824782D78023B5B10D5
:101D3000641B63435201B2E72378DBB2B2E70228A7
:101D4000D5D11D4B1B78013B022B03D91B4B1B78B4
:101D5000022BCCD16C20C8E79809FF1FFC0FFF1F96
:101D60005066FF1FFF3F0000141003405466FF1F22
:101D70000C10034000100340D50BFF1F7211FF1F12
:101D8000B40003408C09FF1F680AFF1F490AFF1FA8
:101D900094000340460AFF1F470AFF1FF908FF1F70
:101DA0002209FF1F300DFF1F3409FF1FBC0BFF1F4F
:101DB000440AFF1F450AFF1F1C09FF1F2309FF1FBD
:101DC00010B502F07DF80022014B1A8010BDC0460C
:101DD0004C66FF1F10B502F03BF9A121054A8900AE
:101DE0009478054A61431268044B5218528C1A8049
:101DF00010BDC046300DFF1F3409FF1F4C66FF1F8A
:101E000010B50D4B0D4A9978A1239B004B431268E6
:101E1000D218531DD97F0A4B1B88994209D2441C02
:101E200007D0C82805D0D2695B1A5A43054B5343E3
:101E3000C01802F0B5F810BD300DFF1F3409FF1FA8
:101E40004C66FF1F7102000070B5244D2B68002BFB
:101E500028D001F09DFF2B68D8402B680400002B90
:101E600027D002F025F82B68D8401D4B1D4A9978E1
:101E7000A1239B004B431268D118D25C91239B0095
:101E8000002A20D0CA580132CA50174B17491B6884
:101E90000868834214D3D23B181A012A1AD0144B73
:101EA000186070BD01F074FF124B196802F080F8E1
:101EB000D3E701F0FDFF0F4B196802F079F8D4E782
:101EC0000D495B18E8E7CA500C4B1B68DB68E41847
:101ED000201AE4E7F530FF30E1E7C0461C08FF1F99
:101EE000300DFF1F3409FF1F9C09FF1F5066FF1FA5
:101EF000A009FF1F1808FF1F2DFF3F005866FF1F96
:101F000070B504000D00282916D10300A433C2883F
:101F10001B889B1A0B4A9BB293420DD906006A3666
:101F200005223100653002F033F8002804D1310079
:101F3000200001F015FF70BD2900200002F098F884
:101F4000F9E7C046FE7F0000F8B50400012001F06B
:101F500087FF01F0EDFE174A17491060096803007A
:101F60001648174E01601748776805680020AF4291
:101F700001D27068281A144D091928601348C162EB
:101F8000A421446A49032143416211490978002987
:101F900005D010490978022902D10F3B1360F8BD22
:101FA000012901D1083BF9E7032901D1053BF5E7F8
:101FB000033BF3E7E408FF1F28F00040340AFF1F4B
:101FC00028100040180AFF1F1C0AFF1F00F00040E5
:101FD0001C09FF1F4A0AFF1F70B580241025E40565
:101FE000A3682B43A36001F0CBFEA368AB43A360BF
:101FF00070BD0000F7B5160080221C001023D2052A
:102000000191916805000B43936000225A4BD73031
:102010001A6001F0CDFE9D232A002F009B00EB5893
:10202000CA3201210092FC37002B01D00021009A16
:10203000386802F015F82900009BCB311A784F4B15
:10204000D3351A604B780A781B0213438A7812043E
:102050001A43CB781B061343494A1BBA13604B79CA
:102060000A791B0213438A7912041A43CB7931008F
:102070001B061343434A1BBA13606B782A781B0272
:102080001343AA7812041A43EB781B0613433E4A03
:102090001BBA1360019A330213433C4A13603C4B52
:1020A00022001B1B9C4603293DDCB3089A00130049
:1020B0005142B21A032A46D1354AE018511A8278A1
:1020C0004078120400020243E05C043302430A60D9
:1020D0000022FF2B4BDDF0222E4B12011A600F2243
:1020E0002D4B1A602D4A1368002BFCD00023224A86
:1020F00027491360091B321D0B191B68043A180A83
:1021000023706070180C1B0EA070E3700434002A5A
:10211000F2DC802210213B68D20501333B609368DA
:102120008B439360F7BD6346D578981893782D0656
:102130001B042B43157804392B43557804322D02A8
:102140002B430360AFE7022A0AD1114AE05C511A1F
:10215000E2185278120202430A6004339BB2B7E7D6
:10216000012AB5D10A4A521AE15C1160F5E7084923
:1021700059180A600433ACE7000004403C000440F6
:102180003800044034000440300004400C00044097
:102190000001044004000440100004401400044006
:1021A000F7B5150080221C001023D205009191681C
:1021B00007000B4393600023654AD730136001F09A
:1021C000F7FD9D233E009B00F9583B00CA363200C4
:1021D000FC33002900D07FE0586801F041FF39004E
:1021E00032785C4BCB311A604B780A781B02134370
:1021F0008A78AC4612041A43CB78281D1B06134379
:10220000554A1BBA13604B790A791B0213438A792A
:1022100012041A43CB791B061343504A1BBA1360AE
:102220004B7A0A7A1B0213438A7A12041A43CB7A36
:1022300021001B0613434A4A1BBA1360009A2B0263
:102240001343484A13602200474B1B1B0093009B1B
:10225000CE785B1801938B7836061B0433430E78D7
:10226000043833434E78043136023343019E3360E1
:102270000328ECDC0321A808431C9B0029408000B4
:1022800003292BD13849E5185E18A9786D78E35CED
:1022900009042D022943194331600300083300214A
:1022A000FF2B2DDD314B324919600F21314B196065
:1022B000012327490B60304B19680029FCD0062107
:1022C0001B680B40042B20D080220020D20593688D
:1022D0000A318B439360FEBD01217DE7022908D1BD
:1022E00021495D18E1184978E35C09021943296026
:1022F000D3E70129D3D11C495918E35C0B60CCE723
:102300001948181801600433CAE7002310490B600C
:102310006346002B0CDC3B00FC335A681021013271
:102320005A608022D205936801208B439360D2E7E4
:10233000009B9B181B68190A13705170190C1B0E17
:10234000D37004235B4291709C440432E0E7C046A2
:10235000000004403C0004403800044034000440C5
:10236000300004400C00044000010440040004401C
:10237000080F0000100004401400044070B5061E51
:1023800019D00222614B9B799343012B13D1604BEF
:102390001A78FF2A0FD15A78FF2A0CD19A78FF2A8F
:1023A00009D1DA78FF2A06D11A79FF2A03D15B799D
:1023B000FF2B00D1A7E0574B0C201A78012A08D038
:1023C0000022554D1A702B781A00093A042A01D8B8
:1023D000212070BD5A1F012AFAD94C4CA07B042839
:1023E00000D990E0A279032A00D98CE0821E012A4C
:1023F00003D862881F2A00D885E0002E61D0012E04
:1024000000D080E0A288012AE2D0002B0AD1013856
:10241000032803D801F066FC151D19151F202E7026
:1024200001F086FD2B785A1E032A16D800253B4B57
:102430001D602823237501F043FEA8422ED0A580FD
:10244000C6E7022320202B70EAE7042322202B700A
:10245000E6E7032321202B70E2E7073B012BB7D8E7
:102460002F4B1B68DB6A9B06B2D52E4B1A78002ACD
:10247000AED1A27B911E012901D9002AA8D1022246
:1024800080211A702823284D89012878237501F0AE
:102490002FFE80212878890101F03AFC0123A380D6
:1024A000224B1B78002B0AD0FA228021204B92006D
:1024B0001B8809025A431C4B187801F051FD00207B
:1024C00087E701F03DFE2B78A680073B012B06D95C
:1024D00018482E7001F0ACFE1E2001F029FD114BB2
:1024E000114C1A78002A06D0802100222078890118
:1024F0001A7001F0FDFD01F063FE802120780902D1
:1025000001F0F6FDDBE7122063E7C046A60BFF1FD4
:102510006B09FF1F1A09FF1F1C09FF1F4809FF1F36
:102520005866FF1F2309FF1F1B09FF1F2109FF1FFB
:102530002C09FF1F0010004010B5002901D001F048
:1025400067FC10BDF7B5604B01919978A1239B0002
:102550004B435E4A060014681022E418D6235B0041
:10256000E0583623FF33E35C00279343222B41D10D
:10257000574B0F3A1A600760012501F069FE019B75
:102580001880E8235B00E35C002B01D0B34258DDE8
:102590000023504FFB70AD33FF33E3581A68002A15
:1025A00003D09B88DB439B071DD03823FF33E35CBC
:1025B000002B18D09B235B00E35C002B13D1D1339D
:1025C000FF33E35CB3420EDAA4235B00E15AE01868
:1025D000090A023101F054FC23000122FE33013EBE
:1025E00001351A87FA70E8235B00E35C002B2AD0E0
:1025F000A8B2FEBD03683D00002BBED08188043028
:10260000090A023101F03CFCD6235B00E3581F604D
:10261000B2E72300B133BA00FF33985801378188FD
:102620000430090A023101F02BFCE8235B00E35C73
:10263000BB42EEDCE822F61AED1800235200A35448
:10264000A6E70027F1E7200001F052FC00281FD088
:10265000002E1DDD7319882647190193B60020004E
:1026600001F0C6FB5A30800020184068013581888F
:102670000430090A023101F003FC200001F010FDD2
:10268000A3590133A351BD4202D0019B9D42E6D123
:10269000114BE35C002BABD095239B00E35C002B3C
:1026A000A6D00E4BE15A0029A2D00D4AA35C994254
:1026B00002D90133A3549BE700231A212000A3541D
:1026C00001F08EFD94E7C046300DFF1F3409FF1F57
:1026D00000140340E010FF1F5A02000072020000C5
:1026E0005E020000F8B51D4B1D4F1A78002A10D16C
:1026F000BA7B002A02D101321A7003E0032AFAD011
:10270000022AF8D001F0DCFC00220120154B1A70DF
:10271000F8BD154B154D1C68154B9E7801232B7089
:102720002878C0B200F0DEFCBB7B002B0BD101F09F
:102730004FFBA1239B007343E41883239B00E41801
:1027400023782B70E4E7032B02D101F069FCF0E75A
:102750000020022BDCD101F0D3FBEAE71C09FF1FAC
:10276000A60BFF1F2309FF1F3409FF1F490AFF1F84
:10277000300DFF1FF0B587B00EAD2F780FAD2D785F
:102780000593AC46634614000E4D0CAA12782E78C1
:1027900003930D9B009201932200059B029701F089
:1027A000F7FC2E70012C01D0042C08D180220649A0
:1027B0008B889343054A1278D20113438B8007B06C
:1027C000F0BDC0461C09FF1F6C11FF1F7809FF1FD9
:1027D0000B001B3B70B504003020E02B0DD813001C
:1027E000E025493BFF3B9BB2ED00AB4205D8034BD4
:1027F000200019825A8201F01BFB70BD8410FF1F5C
:1028000010B501F0B5FA054B00205B68052B04D923
:10281000034A5268D20200D4980810BD001000404C
:10282000FCE100E070B501F08BFC0D4B1B68FC3344
:10283000DC691D6AFFF7E4FF6419844204D2094B86
:1028400001241B68002B07D004220024064B1A70B9
:10285000064A93690133936101F0B2FC200070BD18
:102860005866FF1F9809FF1F2309FF1FFC0FFF1F5A
:1028700070B50C4D2B68FC335C6A01F061FCFFF70E
:10288000BFFF2B680025FC339B6AE318834204D208
:10289000054B1B68AB4200D1051B01F091FC2800E1
:1028A00070BDC0465866FF1F9809FF1FD722044B12
:1028B00092009B5810B5002B00D0984710BDC04621
:1028C0000000FF1FF0B587B001F096F9FFF7EEFFAB
:1028D000CA4BCB4C04931B78022B45D1C94B1B68C8
:1028E000186A01F0BDFAC84BC84A1A60C84BC94AF9
:1028F0001A60A022C84B52001A60049B187801F09D
:102900004FFCC649C64801F08BFAC649C64801F0DB
:1029100087FA1022C54BFF201A60802252031A60EA
:10292000802292031A60802212041A6001F018FCBF
:10293000012001F0FDFBFA20400001F0F1F95820E0
:1029400001F0FEFABA4801F013FB012001F000FB90
:10295000072001F065FC2268B64B1A4084235B0017
:102960001343236007B0F0BD01F092FAB24E02901B
:10297000322001F075FA33681B0629D43C2001F09F
:102980006FFA0F2001F06CFA9C4B1B78012B00D1E1
:102990001EE180223368A94D134200D0A7E02B68C6
:1029A000032013432B6001F05BFA01F071FA029BE4
:1029B0000299C31A5A1E814200D81A00A04B1A600D
:1029C000904B19681E2353439E4A9B18CB618AE79C
:1029D00001F05EFA80239C4ADB02116803900B43EE
:1029E00013602268934B994F1A40282313432360A6
:1029F000032001F035FA03203D6801F031FA3B680D
:102A00000320DB03DB0B009301F02AFA3B68ED03A4
:102A1000DB03ED0BDB0B8E4A0193AB18C22B30D8D6
:102A2000009B9B18C22B2CD8019B9B18C22B28D82B
:102A3000009B2A009D4200D21A00009B9D4200D9B3
:102A40001D00019B934200D21300019A954200D9C8
:102A500015005B1B122B14D80C22336814209343EF
:102A6000336033687B4A1340336001F0F9F9082181
:102A70003B682268DB038A432260774ADB0B1360E2
:102A80007FE7032001F0ECF93B68DB03DB0B0593E8
:102A900001F0FEF9039B0399C21A531E814200D82C
:102AA00013006E4A93421BD9FF23356869492D0AEA
:102AB0001D4032686B1C1B060A401B0C134333601D
:102AC0000C23326800209A43083B1343336001F023
:102AD00007FA6348634BA840984206DCFEF732FFD2
:102AE000019B009D0093059B95E75F48F6E7002357
:102AF0005E4F554A3B6080231168DB020B43136035
:102B000080222B68032013432B6001F0A9F93B6856
:102B1000052601333B6080232A685B0213432B6048
:102B20002268444B03201A40514B1343236001F0A9
:102B300097F90821454B1A682368D2038B43236019
:102B4000454B023900931B68D20B4B439A420CD879
:102B50009B1A3B2B0BD8236846490B4023602B68FC
:102B60000B402B60444B1A601FE7D31AF1E7013E7C
:102B7000F6B2002ED4D123683E4A134023602B685E
:102B800013402B603B68042B07D9BFF34F8F3B4B9F
:102B90003B4ADA60BFF34F8FFEE780222B680320A9
:102BA00093432B6001F05CF92268224B03201A400A
:102BB00028231343236001F053F9244B009A1B6828
:102BC000DB03DB0B1360082223689343236097E742
:102BD00007222C4D2B681340012B02D1002001F05D
:102BE000DFFAAB68284A02201340AB6001F038F9E5
:102BF0008023AA685B001343AB60D6E64A0AFF1F36
:102C00005CF000405866FF1F000003400180063D55
:102C1000BC00034034080000A4000340710200001F
:102C200014100040FFFF3F002810004000E100E0CA
:102C30003075000000FEFEFFC4F0004044F000408C
:102C40004066FF1F7206000040F0004064F0004044
:102C500091FCFFFFFF00FFFF4866FF1FE30C000031
:102C6000E88000005F361E0060361E00B444FF1F7F
:102C700028000100FFFFFEFF4466FF1F00ED00E09B
:102C80000400FA053CF00040FFFEFFFF694E336888
:102C900088331B6883F3088801F022FA00F014FCE3
:102CA000654B664A1B68934207D0002001F018F973
:102CB0000221634A13688B431360FFF703FE614BE5
:102CC000614C1878C0B201F08BF90023A360023385
:102CD000A3605E4B0120236001F0C2F80323A360D0
:102CE00001F0D6F8040001F043F8050001F0D0F837
:102CF000574B186001F07CFA564B1968621A531E44
:102D0000A14200D213008022D203934201D39B023E
:102D10009B0A3268D16AC90700D478E04E491C0C7E
:102D200009689BB24C4359432402090A64180327DB
:102D30004A49FC3293680A6849489B1A494A4A4EF4
:102D400012684A499B18414A34609A183B400193E3
:102D5000036892089C46019B0A6063440360042B4D
:102D600003D901323B400A6003600B684049E41814
:102D7000200001F01DF93F4F3D493B68C3183B60FF
:102D80002000019301F044F93B4C206808183849B1
:102D90002060884205D9019B01333B6001F038F97E
:102DA000216001F045F9354B1B78002B0ED000F067
:102DB000DFFF3168324B4A1B1B6812189A4233D22C
:102DC000591A4919091A2F4801F02AF82E4C237A6A
:102DD000002B0FD000F0CCFF3168E3684A1B1218BB
:102DE000934224D9591A4919091A284801F018F8A8
:102DF00000232372264B83F3088801F0E1F80220B8
:102E000001F096F8002001F06BF800F0D9FFDC012A
:102E100099000234641A5900641A09214B43803323
:102E2000CB40A408E41882E7FA218900CBE71949CE
:102E3000DBE7C0465866FF1F0C0AFF1FB64121039F
:102E400010000040490AFF1F14100040C409000090
:102E5000100AFF1F340AFF1F380AFF1F200AFF1F36
:102E6000280AFF1F1C0AFF1F3C66FF1F240AFF1FC2
:102E7000710200006008FF1F2C0AFF1F1C09FF1FC2
:102E8000E408FF1F00100040740BFF1F3C100040BF
:102E900000000020DC050000A022054B92009B589A
:102EA00010B5002B01D0984710BD01F0B1F9FBE738
:102EB0000000FF1FA122054B92009B5810B5002B6C
:102EC00001D0984710BD01F0A3F9FBE70000FF1FF8
:102ED000A222054B92009B5810B5002B01D09847B9
:102EE00010BD01F095F9FBE70000FF1FA322054B81
:102EF00092009B5810B5002B01D0984710BD01F0EF
:102F000087F9FBE70000FF1FA422054B92009B58A6
:102F100010B5002B01D0984710BD01F079F9FBE7FF
:102F20000000FF1F70B500F023FF514B1860042014
:102F300000F0FEFF01F0ECF80400C30702D401F03A
:102F4000C7F870BD00224B4B1A604B4B1878013804
:102F500004282CD800F0C6FE03231B1F27002000E6
:102F600000F0F6FE0128ECD0444C2378042B71D1FC
:102F700001F066F9002806D001F002F9582000F0AF
:102F8000DFFF02232370032000F0D2FFD9E72000E7
:102F900000F006FFE6E7200000F05AFFE2E720001D
:102FA00000F0BEFFDEE7200001F0BAF8DAE700F03B
:102FB0005FFF0500012808D1314B1B78053B012B31
:102FC00003D82000FFF768FFCEE72C4B1B78022BBD
:102FD00001D0052B20D1022D28D12A4B9B7BAB435E
:102FE0001CD12000FFF766FF254B18780128BBD1C4
:102FF0006405B9D4234925224B7B034205D1233AEA
:1030000013405A42534126331A000B7D9342ABD9E9
:10301000322001F04DF8A7E7022D07D1184B1B789D
:10302000052B11D12000FFF753FFDDE7012D0BD158
:10303000012B03D12000FFF759FF95E7062B03D1A1
:103040002000FFF761FF8FE7200001F0E1F8022D7B
:103050008AD1C9E7032B04D10B4B987C01F088F887
:1030600091E7072B8FD1094B987B01F049F88AE74C
:103070009C09FF1F9809FF1F9009FF1F2309FF1FCD
:103080001C09FF1FA60BFF1FBC0BFF1FD40BFF1F4C
:10309000FA210A4B0A4A49001A640A4A5A500A4A53
:1030A00004395A50094A08319A64094A5A50094A5F
:1030B0005C315A50084ADA667047C0460000FF1F6C
:1030C0007527FF1F7128FF1F2528FF1F7D23FF1F66
:1030D000E526FF1F011EFF1FD51DFF1F10B500F0C5
:1030E000E9FD10BD8023F7B59C46264B264F019382
:1030F0002649274A274D284C284B02281AD16046DA
:1031000038600868264E3040802636033043086019
:1031100001990978002909D11660224A2A60224AB9
:103120002260E02219689143A03A1BE08021C90285
:103130001160F2E766463E600F68194E3E408027F8
:10314000FF023E430E600199097800290DD11760F6
:1031500001280ED1154A2A60154A2260E02219681A
:103160009143C03A0A431A60F7BD80218902116079
:10317000EEE7E0210F4A02432A600F4A22601A68F4
:103180008A43F0E74B0AFF1FE0000340D8000340EA
:103190009000034000000340500003404000034003
:1031A000FFFFE3FF0280063D804508220180063DC7
:1031B000806608220080069880550822F8B51E4BCC
:1031C00080261A68002014003440324232D11A6836
:1031D0001A4F32431A6001223B68063093433B602A
:1031E00000F03EFE0122164D2B681E432E603B6808
:1031F0000A2613433B608027BF00124B1B683B42EB
:1032000011D1013EF6B2FF2E09D17E220E4B1C6871
:103210002B68E40B1440934323432B6005E0082004
:1032200000F01EFEE9E7002EEFD180222B68600837
:1032300093432B60F8BDC046C4F000405CF00040F2
:1032400018F0004068F0004060F0004010B500F059
:103250007FFF01215820034A00F0F2FDFFF7AEFF87
:1032600010BDC046600AFF1F10B578220021034838
:1032700000F02EFE00F0ACFF002010BD6069FF1FC3
:1032800070B5040000F05CFF00230C200B4A010025
:1032900059438D18515C00290DD0A14208D101235A
:1032A00000246B7000F0ACFD00F08AFF200070BDC0
:1032B00001330A2BEBD11224F6E7C0466069FF1FE9
:1032C00070B5040000F03CFF002319001D000D4AFA
:1032D0001078002806D0A0420CD1557001310C3274
:1032E0000A29F5D1002B0AD100F072FF00F068FF27
:1032F000002070BD5078461EB0411B18EEE700F06C
:103300007FFDF3E76069FF1FF7B504000C20002381
:1033100084460E4D019267465F43E85D7E19A042E8
:1033200012D000280BD10A4B9C4662461B7808330A
:103330001370019B70707C557160B360FEBD0133EA
:103340000A2BE8D10320F9E70720F7E76069FF1FA0
:103350005C69FF1F8021F8B5464BC9051B68C12475
:103360008B60454BFF261A68012313434B61434B87
:10337000A4001A68424B40201A60424B1A68424B24
:103380001A60424B1A59B2431A51C52292009D58F5
:10339000B5432843802598509F583D48ED0107408C
:1033A0003D439D509D5880272D022D0A2943995059
:1033B00080211A59090202400A431A5104341A5949
:1033C000344D3F042A403A4380271A511A593F0688
:1033D0001202120A3A431A5108341A5902400A4397
:1033E0001A51C32292009D58B5432C0080252C43CE
:1033F0009C509D582C0004400C439C509D58254CDB
:1034000025408024240425439D509C588025240277
:10341000240A3C439C50C424A4001A59B2432A43B2
:103420001A511A591202120A17431F5108341A5915
:10343000B24315431D5100251A5902400A431A513F
:1034400004341A59024011431951134C134B1B7881
:10345000DB08AB4201DC0020F8BD2378002B06D04E
:10346000A368002B00D0984701350C34EEE71220FA
:10347000F2E7C0464C45FF1F4845FF1FB0F0004033
:103480005869FF1FB4F000405469FF1F00E100E0DD
:10349000FF00FFFFFFFF00FF6069FF1F5C69FF1F68
:1034A000030010B51F2809D8072200201340072465
:1034B00004490A78A24313430B7010BD0023062071
:1034C000F5E7C0465C69FF1F034A04491368002002
:1034D0000B4013607047C0461CF00040FFFFC1FF67
:1034E000054B06491B780A6805485B0702401B0B21
:1034F000134300200B6070475C69FF1F1CF0004005
:10350000FFFFC1FF70B50C25FFF7EAFF0A4B1C78DF
:103510000A4BE4086543ED18002C01D1200070BD72
:103520002B78002B06D06B68002B00D09847013C0D
:103530000C3DF1E71220F2E75C69FF1F5469FF1FA1
:1035400007B50422074801A900F034F9019B0133B3
:1035500005D18023044ADB0411680B43136000206B
:103560000EBDC0461C18001114F00040F0B5050057
:103570002026184B87B00493049B002B03D1112401
:10358000200007B0F0BD002102220B000191009144
:10359000052000F025FC02230F490A681A42FCD1DD
:1035A0000596059C631E0593002CFAD10B4A1368FF
:1035B000002BFCDA0F276F440121380000F008FDD2
:1035C0003B782B42DCD0052000F04AFC049B013BF9
:1035D0000493D1E7FFFFFF0790C8004000C80040F8
:1035E00007B500F0ADFD80220821D205936A019154
:1035F000002B01D10739916202210C4A1160019917
:10360000481E01900029FAD1033111600531019162
:103610000199481E01900029FAD11160002B02D1B6
:103620008022D205936200F0CBFD07BD00C00040B0
:10363000F0B52D4C89B02378002B4FD1FEF762F9FD
:1036400002232A4F03903A681A42FCD120230693A2
:10365000069B5A1E0692002BFAD1254E3368002B8A
:10366000FCDA0120FFF782FF011E02D0112009B011
:10367000F0BD030003220190009005AD9F2000F0F3
:10368000AFFB0321280000F0A3FC02233A681A4292
:10369000FCD120230793079B5A1E0792002BFAD1D7
:1036A0003368002BFCDA0120FFF760FF0028DDD132
:1036B0000398FEF73BF9AA786B7811041B020B43C1
:1036C00029780B4363601300113B0A49052B07D887
:1036D00001239340A3600B60012323700020C6E701
:1036E00080231B03F6E7C0463445FF1F90C8004007
:1036F00000C800409808FF1F1E4B30B55A68187864
:103700001D4B85B0D31859424B4101210093002332
:1037100000F036FC194B1A4A02259A6300221A65FA
:1037200010325A658022C4219D65164B1648D2027C
:10373000DA6789004258154B80241A4080231B0405
:1037400013434350642341200393E40500F078F9C8
:10375000402000F075F96562039D6B1E0393002DF8
:10376000FAD103236362FFF73BFFA562FFF760FF17
:1037700005B030BD4045FF1F95FFFEF700C8004073
:10378000050001FF04E100E000E100E0FFFF00FFB1
:1037900010B5064B18705960FFF7AEFF00211320DB
:1037A000034AFFF7B1FD002010BDC0464045FF1F92
:1037B000F936FF1FF0B5040085B003920291FEF7C1
:1037C000A1F8882263035B0B52051A438023DB05B3
:1037D0009D6A8023274F0092BA68002601901B0340
:1037E0009A420CD9F82326001B041E401C4206D026
:1037F0008022214B52025E6219680A431A60002D32
:103800000BD100F09DFC02221C4B1A608023DB05CB
:103810005A62013A9A6200F0D3FC0023039A934261
:1038200020D1002D0AD100F08BFC144B03221D6027
:103830008023DB055A629D6200F0C2FC8023BA68D7
:103840001B039A4208D9002E06D000220A4B0C49CD
:103850005A621A680A401A600198FEF767F8002059
:1038600005B0F0BD009A0299D2181278CA540133FB
:10387000D4E7C0463445FF1F00C8004000C00040E8
:10388000FFFFFEFFF0B587B0029103920400FEF740
:1038900039F8019000F054FC802302250122234EC8
:1038A000DB0535605D629A6200F08AFC204F3B6860
:1038B0002B42FCD120230493049B5A1E0492002B1C
:1038C000FAD11C4D2B68002BFCDA0120FFF74EFECD
:1038D000002802D0112007B0F0BD2000039A029901
:1038E00000F066FC022304003A681A42FCD120234F
:1038F0000593059B5A1E0592002BFAD12B68002BCD
:10390000FCDA0120FFF732FE051EE3D100F018FCBF
:1039100080230322DB0535605A629D6200F050FC73
:103920000198FEF703F8E0B2D5E7C04600C00040BA
:1039300090C8004000C80040F0B5802687B0040061
:10394000FDF7E0FFF605B36A02250393029000F04D
:10395000F7FB0123244F3D607562B36200F030FC39
:10396000224E33682B42FCD120230493049B5A1E21
:103970000492002BFAD11E4D2B68002BFCDA01209B
:10398000FFF7F4FD002802D0112007B0F0BD2000A1
:1039900000F036FB0223019032681A42FCD120234A
:1039A0000593059B5A1E0592002BFAD12B68002B1C
:1039B000FCDA0320FFF7DAFD041EE5D100F0C0FBBE
:1039C00080230322DB053C605A629C6200F0F8FB16
:1039D000039B002B01D1FFF703FE0298FDF7A6FF22
:1039E0006B461879D1E7C04600C0004090C800403F
:1039F00000C8004007B5000201910422000A01A995
:103A0000FFF740FF0EBD000073B5050005240B4A0B
:103A1000A3005B429B1819686B46DE1D300000F066
:103A20002FFB022804D133782B55013CEFD276BD11
:103A3000052CFCD00128FAD10230F8E71409001156
:103A40001F2807D8012380228340D20591680B43A9
:103A5000936070473F2808D8012380222038834094
:103A6000D20551690B435361F3E75F28F1D8012375
:103A7000802240388340D205116A0B431362E8E785
:103A80001F2807D8012280218240C9058B689343F3
:103A90008B6070473F2808D801228021203882405F
:103AA000C9054B6993434B61F3E75F28F1D80122C5
:103AB000802140388240C9050B6A93430B62E8E7D6
:103AC0001F2810D880230200DB05153A1968012A47
:103AD00006D820229143196019680A431A6070477A
:103AE00001228240F6E73F2811D880230200DB053F
:103AF000353AD968032A06D810229143D960D9688B
:103B00000A43DA60EBE7012220388240F5E75F28BC
:103B1000E5D842238022181A413B8340D205516ADE
:103B200099435162516A0B435362D8E710B50400C0
:103B3000012813D1A022184992050B685B015B098B
:103B400013430B60154B164A19681140154A0A4376
:103B50001A60402219680A431A6010BD0028FCD17F
:103B600001000A2000F0ECF821000B2000F0E8F83A
:103B7000C0220A4B920019680A4340211A601A6851
:103B80008A431A60B022044912060B685B015B0984
:103B900013430B60E1E7C04614F000401CF0004006
:103BA0007F00FEFF80FD010072B6074A13680133F3
:103BB00013600422054B1A600023054A136080221B
:103BC000D2055360FEE7C0467808FF1FC0F00040F2
:103BD000C4F00040044B054A1A60054B1A600022ED
:103BE000044B1A607047C046140AFF1F841E000071
:103BF000380AFF1FC4F000400023034A1360034A41
:103C00001360034A1360704754F0004040F10040D5
:103C100044F10040002310B5184C8AB00093019382
:103C20002378012B27D06946012000F0E9FA00280B
:103C300017D1009B12490293019B06AA0393114BD3
:103C400002A81B680493104B1B68059300F098F8BA
:103C500010220E4906A800F09BF9002804D1FF238A
:103C6000237000200AB010BD0123094A074902A8A9
:103C7000237000F085F80120F4E7C0465C66FF1F62
:103C800010290011082900110C2900112029001108
:103C90006066FF1F13B501246946012000F0B0FAE9
:103CA000034B00940193FFF7B5FF200016BDC046FB
:103CB000BB0B000010B5FFF79FFFFFF7EBFF0028DD
:103CC00002D0024B984710BDFEE7C046E1A20000BB
:103CD00002B4714649084900095649008E4402BCA5
:103CE0007047C04602B4714649084900095C490062
:103CF0008E4402BC7047C04603B471464908400078
:103D00004900095A49008E4403BC70470000000076
:103D100001B40248844601BC604700BF0D52010057
:103D200001B40248844601BC604700BF851201000F
:103D300001B40248844601BC604700BFBD5C01007D
:103D400001B40248844601BC604700BFED9E0011EB
:103D500001B40248844601BC604700BF0134010041
:103D600001B40248844601BC604700BF85C1000021
:103D700001B40248844601BC604700BFC95C010031
:103D800001B40248844601BC604700BFDD3F00002B
:103D900001B40248844601BC604700BFE90B010042
:103DA00001B40248844601BC604700BF09340100E9
:103DB00001B40248844601BC604700BF894400004A
:103DC00001B40248844601BC604700BF855201002F
:103DD00001B40248844601BC604700BFE9F6000018
:103DE00001B40248844601BC604700BF496D010030
:103DF00001B40248844601BC604700BFD9B000004E
:103E000001B40248844601BC604700BF21A90000FC
:103E100001B40248844601BC604700BFE9D40000F9
:103E200001B40248844601BC604700BF2D6C01000C
:103E300001B40248844601BC604700BF116E000017
:103E400001B40248844601BC604700BF016701001D
:103E500001B40248844601BC604700BF053401003C
:103E600001B40248844601BC604700BF01890000DC
:103E700001B40248844601BC604700BFDD0C01006C
:103E800001B40248844601BC604700BFC11501006F
:103E900001B40248844601BC604700BF156B0100B5
:103EA00001B40248844601BC604700BFE927000016
:103EB00001B40248844601BC604700BF6D0B01009D
:103EC00001B40248844601BC604700BF8D820000F7
:103ED00001B40248844601BC604700BFB70E000031
:103EE00001B40248844601BC604700BF016C010078
:103EF00001B40248844601BC604700BF71B00000B5
:103F000001B40248844601BC604700BF19FA0000B2
:103F100001B40248844601BC604700BFA1AF000065
:103F200001B40248844601BC604700BFF53501007A
:103F300001B40248844601BC604700BF1907010074
:103F400001B40248844601BC604700BF79120100F9
:103F500001B40248844601BC604700BFE51201007D
:103F600001B40248844601BC604700BF8B52010087
:103F700001B40248844601BC604700BF8D110100B6
:103F800001B40248844601BC604700BFC56D010012
:103F900001B40248844601BC604700BFCD4C01001B
:103FA00001B40248844601BC604700BF8937010064
:103FB00001B40248844601BC604700BF090E0000FE
:103FC00001B40248844601BC604700BF79970000F5
:103FD00001B40248844601BC604700BF3D71010046
:103FE00001B40248844601BC604700BF8914010047
:103FF00001B40248844601BC604700BFF9A6000036
:1040000001B40248844601BC604700BFA96F0100AB
:1040100001B40248844601BC604700BF090E00009D
:1040200001B40248844601BC604700BF75F8000037
:1040300001B40248844601BC604700BFD54401007A
:1040400001B40248844601BC604700BFE94C01004E
:1040500001B40248844601BC604700BFF9ED00008E
:1040600001B40248844601BC604700BF21440000FF
:1040700001B40248844601BC604700BF51B800004B
:1040800001B40248844601BC604700BF8D3800116E
:1040900001B40248844601BC604700BFD9B2001198
:1040A00001B40248844601BC604700BF5976010054
:1040B00001B40248844601BC604700BF613701007B
:1040C00001B40248844601BC604700BFA9D8000083
:1040D00001B40248844601BC604700BFDD0A01000C
:1040E00001B40248844601BC604700BFC9A9000072
:1040F00001B40248844601BC604700BFB3520100CE
:1041000001B40248844601BC604700BFC1F700000B
:1041100001B40248844601BC604700BFBD0B0100EA
:1041200001B40248844601BC604700BFF935010074
:1041300001B40248844601BC604700BF6911010018
:1041400001B40248844601BC604700BF75A9000065
:1041500001B40248844601BC604700BFED6801001D
:1041600001B40248844601BC604700BFED6B01000A
:1041700001B40248844601BC604700BF4DF900000D
:1041800001B40248844601BC604700BF6DF60000E0
:1041900001B40248844601BC604700BF9D6A00002C
:1041A00001B40248844601BC604700BFEDA5000091
:1041B00001B40248844601BC604700BF957301000A
:1041C00001B40248844601BC604700BF9DA90000BD
:1041D00001B40248844601BC604700BFADAE000098
:1041E00001B40248844601BC604700BF53B90000D7
:1041F00001B40248844601BC604700BFC1660100AB
:1042000001B40248844601BC604700BFE1AC000035
:1042100001B40248844601BC604700BFE9170100B1
:1042200001B40248844601BC604700BFF90D01009B
:1042300001B40248844601BC604700BFC1A500002C
:1042400001B40248844601BC604700BF01D70000AA
:1042500001B40248844601BC604700BFCD0C010098
:104260000200000012BC001101000000E0B90011C2
:10427000020000000EBC001101000000A042FF1F60
:1042800002000000E8B9001101000000A463FF1F54
:10429000020000000CBC0011030000001863FF1FA7
:1042A000120000000200000012BC0011010000001A
:1042B00028BA0011020000000EBC0011010000002D
:1042C00025BA00110200000032BA001103000000FC
:1042D0005363FF1F020000000CBC0011030000002C
:1042E0006863FF1F020000000EBC00110100000007
:1042F00024BA00110200000030BA001103000000CF
:104300002963FF1F020000000CBC00110300000025
:104310004A63FF1F0200000012BC001101000000F0
:104320006CBA0011020000000EBC00110100000078
:10433000E943FF1F020000007EBA001101000000E7
:1043400063BA0011020000000EBC00110100000061
:10435000E843FF1F020000007CBA001101000000CA
:104360007063FF1F020000000EBC0011010000007E
:10437000E743FF1F020000007ABA001101000000AD
:1043800053BA0011020000000EBC00110100000031
:10439000E643FF1F0200000078BA00110100000090
:1043A0004EBA0011020000000EBC00110100000016
:1043B000E543FF1F0200000076BA00110100000073
:1043C00049BA0011020000000EBC001101000000FB
:1043D000E443FF1F0200000074BA00110100000056
:1043E00044BA00110202020202020000B54B0011A1
:1043F000794B0011C0BA0011900118001800FFFF9E
:104400000701020304050602010600000000000087
:10441000000000000000000000000000000000009C
:1044200000000000000003000200000012BC0011A8
:104430000100000040BB0011020000000EBC001192
:10444000010000009844FF1F020000004ABB001159
:10445000010000009E63FF1F020000000CBC001161
:10446000030000000C66FF1F020000000EBC0011DC
:10447000010000009844FF1F0200000048BB00112B
:1044800001000000A063FF1F020000000CBC00112F
:10449000030000000466FF1F12000000000100007E
:1044A00000000111FFFF00005048593600000000D5
:1044B0000000000001000000D1BA00110B0005004F
:1044C000F7000000B4000028002800283075A00084
:1044D000A000A000A00000080008E001F00010000B
:1044E000100010001000100010005000500050008C
:1044F00010001000D0070000000000000F000100B5
:104500000500307507001000010081FF0000000069
:10451000FF000000D5700011DD6E00116D6C001100
:10452000FFFF0100FF000000F19A00116D980011DB
:104530008597001100000000000000000000080046
:10454000040000003B0001085902E0018821280016
:10455000FF0000000200000012BC0011010000007A
:10456000D8BC0011020000000EBC001101000000C8
:10457000D145FF1F020000000ABC0011010000002D
:10458000186AFF1F020000000EBC001101000000AD
:10459000D045FF1F0200000008BC00110100000010
:1045A000CE45FF1F020000000EBC001101000000FC
:1045B000CC45FF1F0200000006BC001101000000F6
:1045C000C445FF1F180018000000900102000003FE
:1045D000020200000200000012BC001101000000F5
:1045E000ECBC0011020000000EBC00110100000034
:1045F0001446FF1F0200000004BC00110000000070
:1046000000000000020000000CBC001103000000CC
:06461000386AFF1F20FFC5
:040000051FFF184180
:00000001FF
